 M1

 Timestamp is 338e06ff (Thu May 29 18:45:19 1997)

 Preferred load address is 00400000

 Start         Length     Name                   Class
 0001:00000000 00016224H .text                   CODE
 0002:00000000 00005ae4H .rdata                  DATA
 0002:00005ae8 000005a8H .xdata$x                DATA
 0002:00006090 00000000H .edata                  DATA
 0003:00000000 00000004H .CRT$XCA                DATA
 0003:00000004 00000004H .CRT$XCL                DATA
 0003:00000008 00000084H .CRT$XCU                DATA
 0003:0000008c 00000004H .CRT$XCZ                DATA
 0003:00000090 00000004H .CRT$XIA                DATA
 0003:00000094 00000004H .CRT$XIZ                DATA
 0003:000000a0 00000c1dH .data                   DATA
 0003:00000cc0 00010e18H .bss                    DATA
 0004:00000000 00000078H .idata$2                DATA
 0004:00000078 00000014H .idata$3                DATA
 0004:0000008c 00000380H .idata$4                DATA
 0004:0000040c 00000380H .idata$5                DATA
 0004:0000078c 0000031eH .idata$6                DATA
 0005:00000000 00000568H .rsrc$01                DATA
 0005:00000570 0000253cH .rsrc$02                DATA

  Address         Publics by Value              Rva+Base   Lib:Object

 0001:00000000       ?openfile@Bufferinputbitstream@@QAEDPAD@Z 00401000 f input.obj
 0001:0000008c       ?getbytedirect@Bufferinputbitstream@@QAEHXZ 0040108c f input.obj
 0001:000000ef       ?readbuffer@Bufferinputbitstream@@QAEDH@Z 004010ef f input.obj
 0001:0000016c       ?getbyte@Bufferinputbitstream@@QAEHXZ 0040116c f input.obj
 0001:000001c4       ?getbits@Bufferinputbitstream@@QAEHH@Z 004011c4 f input.obj
 0001:000002b0       ??1Rawplayer@@UAE@XZ       004012b0 f rawplayer.obj
 0001:0000032b       ?initialize@Rawplayer@@UAEDPAD@Z 0040132b f rawplayer.obj
 0001:00000390       ?setsoundtype@Rawplayer@@UAEDHHH@Z 00401390 f rawplayer.obj
 0001:000003ea       ?putblock@Rawplayer@@UAEDPAXH@Z 004013ea f rawplayer.obj
 0001:00000420       ??1Soundplayer@@UAE@XZ     00401420 f rawplayer.obj
 0001:00000440       ?getblocksize@Soundplayer@@UAEHXZ 00401440 f rawplayer.obj
 0001:00000460       ??_ESoundplayer@@UAEPAXI@Z 00401460 f rawplayer.obj
 0001:00000460       ??_GSoundplayer@@UAEPAXI@Z 00401460 f rawplayer.obj
 0001:000004a0       ?getblocksize@Rawplayer@@UAEHXZ 004014a0 f rawplayer.obj
 0001:000004c0       ??_GRawplayer@@UAEPAXI@Z   004014c0 f rawplayer.obj
 0001:000004c0       ??_ERawplayer@@UAEPAXI@Z   004014c0 f rawplayer.obj
 0001:00001633       ?computebuffer@Mpegtoraw@@QAEXPAMQAY0CAA@M@Z 00402633 f filter.obj
 0001:00002ac3       ?subbandsynthesis@Mpegtoraw@@QAEXPAM0@Z 00403ac3 f filter.obj
 0001:00002b60       ?generatesingle@Mpegtoraw@@QAEXXZ 00403b60 f filter.obj
 0001:00004a20       ?putraw@Mpegtoraw@@QAEXF@Z 00405a20 f filter.obj
 0001:00004a60       ?generate@Mpegtoraw@@QAEXXZ 00405a60 f filter.obj
 0001:000081e0       ?layer3initialize@Mpegtoraw@@QAEXXZ 004091e0 f mpeglayer3.obj
 0001:00008ccf       ?layer3getscalefactors@Mpegtoraw@@QAEXHH@Z 00409ccf f mpeglayer3.obj
 0001:00009584       ?layer3huffmandecode@Mpegtoraw@@QAEXHHQAY0BC@H@Z 0040a584 f mpeglayer3.obj
 0001:000097f4       ?layer3dequantizesample@Mpegtoraw@@QAEXHHQAY0BC@HQAY0BC@M@Z 0040a7f4 f mpeglayer3.obj
 0001:00009e77       ?layer3reorder@Mpegtoraw@@QAEXHHQAY0BC@M0@Z 0040ae77 f mpeglayer3.obj
 0001:0000a534       ?layer3antialias@Mpegtoraw@@QAEXHHQAY0BC@M0@Z 0040b534 f mpeglayer3.obj
 0001:0000a78d       ?layer3reorderandantialias@Mpegtoraw@@QAEXHHQAY0BC@M0@Z 0040b78d f mpeglayer3.obj
 0001:0000a86c       ?layer3hybrid@Mpegtoraw@@QAEXHHHQAMQAY0CA@M@Z 0040b86c f mpeglayer3.obj
 0001:0000ab1d       ?extractlayer3@Mpegtoraw@@QAEXXZ 0040bb1d f mpeglayer3.obj
 0001:0000b2a0       ?initialize@Mpegbitwindow@@QAEXXZ 0040c2a0 f mpeglayer3.obj
 0001:0000b2d0       ?wgetbits@Mpegtoraw@@QAEHH@Z 0040c2d0 f mpeglayer3.obj
 0001:0000b300       ?gettotalbit@Mpegbitwindow@@QAEHXZ 0040c300 f mpeglayer3.obj
 0001:0000b320       ?rewind@Mpegbitwindow@@QAEXH@Z 0040c320 f mpeglayer3.obj
 0001:0000b370       ?layer3twopow2@Mpegtoraw@@QAEMHHHH@Z 0040c370 f mpeglayer3.obj
 0001:0000b3b0       ?layer3twopow2_1@Mpegtoraw@@QAEMHHH@Z 0040c3b0 f mpeglayer3.obj
 0001:0000b3f0       ?layer3inv_mdct@Mpegtoraw@@QAEXPAM0H@Z 0040c3f0 f mpeglayer3.obj
 0001:0000c160       ?putbyte@Mpegbitwindow@@QAEXH@Z 0040d160 f mpeglayer3.obj
 0001:0000c1a0       ?forward@Mpegbitwindow@@QAEXH@Z 0040d1a0 f mpeglayer3.obj
 0001:0000c1f0       ?getbits@Mpegtoraw@@QAEIH@Z 0040d1f0 f mpeglayer3.obj
 0001:0000c220       ?layer3getsideinfo@Mpegtoraw@@QAEDXZ 0040d220 f mpeglayer3.obj
 0001:0000c570       ?getbit@Mpegtoraw@@QAEIXZ  0040d570 f mpeglayer3.obj
 0001:0000c5a0       ?layer3fixtostereo@Mpegtoraw@@QAEXHQAY1CA@BC@M0@Z 0040d5a0 f mpeglayer3.obj
 0001:0000d300       ?open@Bufferoutputbitstream@@QAEDPAD@Z 0040e300 f output.obj
 0001:0000d34e       ?sync@Bufferoutputbitstream@@QAEDXZ 0040e34e f output.obj
 0001:0000d3be       ?putbits@Bufferoutputbitstream@@QAEDHH@Z 0040e3be f output.obj
 0001:0000d4a0       ?putbyte@Bufferoutputbitstream@@AAEHH@Z 0040e4a0 f output.obj
 0001:0000d4d0       ?Die@MyDsound@@QAEXXZ      0040e4d0 f dsoundctl.obj
 0001:0000d4ee       ?init@MyDsound@@QAEXM@Z    0040e4ee f dsoundctl.obj
 0001:0000dd76       ?writeToDsound@MyDsound@@QAEXPAXH@Z 0040ed76 f dsoundctl.obj
 0001:0000e2ee       ?ValidBufferLeft@MyDsound@@QAEJXZ 0040f2ee f dsoundctl.obj
 0001:0000e364       ?PercentValidBufferLeft@MyDsound@@QAEJXZ 0040f364 f dsoundctl.obj
 0001:0000e3eb       ?Stop@MyDsound@@QAEXXZ     0040f3eb f dsoundctl.obj
 0001:0000e47b       ?SetPriority@MyDsound@@QAEXH@Z 0040f47b f dsoundctl.obj
 0001:0000e540       ??0CPlaylistDlg@@QAE@PAVCWnd@@@Z 0040f540 f PlaylistDlg.obj
 0001:0000e5ba       ?DoDataExchange@CPlaylistDlg@@MAEXPAVCDataExchange@@@Z 0040f5ba f PlaylistDlg.obj
 0001:0000e5de       ?_GetBaseMessageMap@CPlaylistDlg@@KGPBUAFX_MSGMAP@@XZ 0040f5de f PlaylistDlg.obj
 0001:0000e5f3       ?GetMessageMap@CPlaylistDlg@@MBEPBUAFX_MSGMAP@@XZ 0040f5f3 f PlaylistDlg.obj
 0001:0000e610       ??_GCPlaylistDlg@@UAEPAXI@Z 0040f610 f PlaylistDlg.obj
 0001:0000e610       ??_ECPlaylistDlg@@UAEPAXI@Z 0040f610 f PlaylistDlg.obj
 0001:0000e650       ??1CPlaylistDlg@@UAE@XZ    0040f650 f PlaylistDlg.obj
 0001:0000e6b0       ?TimerProc@@YGXPAUHWND__@@IIK@Z 0040f6b0 f M1Dlg.obj
 0001:0000ea2a       ?go@@YAXPAD@Z              0040fa2a f M1Dlg.obj
 0001:0000ed3d       ?play@@YAXPAVCM1Dlg@@@Z    0040fd3d f M1Dlg.obj
 0001:0000f149       ??0CAboutDlg@@QAE@XZ       00410149 f M1Dlg.obj
 0001:0000f1bc       ?DoDataExchange@CAboutDlg@@MAEXPAVCDataExchange@@@Z 004101bc f M1Dlg.obj
 0001:0000f1e0       ?_GetBaseMessageMap@CAboutDlg@@KGPBUAFX_MSGMAP@@XZ 004101e0 f M1Dlg.obj
 0001:0000f1f5       ?GetMessageMap@CAboutDlg@@MBEPBUAFX_MSGMAP@@XZ 004101f5 f M1Dlg.obj
 0001:0000f210       ??0CM1Dlg@@QAE@PAVCWnd@@@Z 00410210 f M1Dlg.obj
 0001:0000f427       ?DoDataExchange@CM1Dlg@@MAEXPAVCDataExchange@@@Z 00410427 f M1Dlg.obj
 0001:0000f55a       ?_GetBaseMessageMap@CM1Dlg@@KGPBUAFX_MSGMAP@@XZ 0041055a f M1Dlg.obj
 0001:0000f56f       ?GetMessageMap@CM1Dlg@@MBEPBUAFX_MSGMAP@@XZ 0041056f f M1Dlg.obj
 0001:0000f58a       ?OnInitDialog@CM1Dlg@@MAEHXZ 0041058a f M1Dlg.obj
 0001:0000f8bb       ?OnSysCommand@CM1Dlg@@IAEXIJ@Z 004108bb f M1Dlg.obj
 0001:0000f94d       ?OnPaint@CM1Dlg@@IAEXXZ    0041094d f M1Dlg.obj
 0001:0000fa68       ?OnQueryDragIcon@CM1Dlg@@IAEPAUHICON__@@XZ 00410a68 f M1Dlg.obj
 0001:0000fa87       ?OnPlay@CM1Dlg@@IAEXXZ     00410a87 f M1Dlg.obj
 0001:0000fc19       ?OnStop@CM1Dlg@@IAEXXZ     00410c19 f M1Dlg.obj
 0001:0000fcad       ?OnDropFiles@CM1Dlg@@IAEXPAUHDROP__@@@Z 00410cad f M1Dlg.obj
 0001:0000fdfb       ?OnFastf@CM1Dlg@@IAEXXZ    00410dfb f M1Dlg.obj
 0001:0000fe11       ?OnRewind@CM1Dlg@@IAEXXZ   00410e11 f M1Dlg.obj
 0001:0000fe27       ?OnSkipb@CM1Dlg@@IAEXXZ    00410e27 f M1Dlg.obj
 0001:0000fe6c       ?OnSkipf@CM1Dlg@@IAEXXZ    00410e6c f M1Dlg.obj
 0001:0000fea5       ?OnOK@CM1Dlg@@MAEXXZ       00410ea5 f M1Dlg.obj
 0001:0000ffd2       ?DestroyWindow@CM1Dlg@@UAEHXZ 00410fd2 f M1Dlg.obj
 0001:00010050       ??0Mpegfileplayer@@QAE@XZ  00411050 f M1Dlg.obj
 0001:000100c0       ??0Fileplayer@@QAE@XZ      004110c0 f M1Dlg.obj
 0001:00010100       ??1Fileplayer@@UAE@XZ      00411100 f M1Dlg.obj
 0001:00010150       ??_EFileplayer@@UAEPAXI@Z  00411150 f M1Dlg.obj
 0001:00010150       ??_GFileplayer@@UAEPAXI@Z  00411150 f M1Dlg.obj
 0001:00010190       ?setforcetomono@Mpegfileplayer@@UAEXD@Z 00411190 f M1Dlg.obj
 0001:000101c0       ?setforcetomono@Mpegtoraw@@QAEXD@Z 004111c0 f M1Dlg.obj
 0001:000101f0       ??_EMpegfileplayer@@UAEPAXI@Z 004111f0 f M1Dlg.obj
 0001:000101f0       ??_GMpegfileplayer@@UAEPAXI@Z 004111f0 f M1Dlg.obj
 0001:00010230       ??1Mpegfileplayer@@UAE@XZ  00411230 f M1Dlg.obj
 0001:000102e0       ??_GMyDsound@@QAEPAXI@Z    004112e0 f M1Dlg.obj
 0001:00010320       ??1MyDsound@@QAE@XZ        00411320 f M1Dlg.obj
 0001:00010380       ??_ECAboutDlg@@UAEPAXI@Z   00411380 f M1Dlg.obj
 0001:00010380       ??_GCAboutDlg@@UAEPAXI@Z   00411380 f M1Dlg.obj
 0001:000103c0       ??1CAboutDlg@@UAE@XZ       004113c0 f M1Dlg.obj
 0001:00010420       ??_ECM1Dlg@@UAEPAXI@Z      00411420 f M1Dlg.obj
 0001:00010420       ??_GCM1Dlg@@UAEPAXI@Z      00411420 f M1Dlg.obj
 0001:00010460       ??1CM1Dlg@@UAE@XZ          00411460 f M1Dlg.obj
 0001:00010610       ??0?$CArray@PAVCString@@PAV1@@@QAE@XZ 00411610 f M1Dlg.obj
 0001:000106b0       ?GetUpperBound@?$CArray@PAVCString@@PAV1@@@QBEHXZ 004116b0 f M1Dlg.obj
 0001:000106d0       ?Add@?$CArray@PAVCString@@PAV1@@@QAEHPAVCString@@@Z 004116d0 f M1Dlg.obj
 0001:00010710       ??A?$CArray@PAVCString@@PAV1@@@QAEAAPAVCString@@H@Z 00411710 f M1Dlg.obj
 0001:00010740       ??1?$CArray@PAVCString@@PAV1@@@UAE@XZ 00411740 f M1Dlg.obj
 0001:00010800       ?Serialize@?$CArray@PAVCString@@PAV1@@@UAEXAAVCArchive@@@Z 00411800 f M1Dlg.obj
 0001:00010890       ?Dump@?$CArray@PAVCString@@PAV1@@@UBEXAAVCDumpContext@@@Z 00411890 f M1Dlg.obj
 0001:00010920       ?AssertValid@?$CArray@PAVCString@@PAV1@@@UBEXXZ 00411920 f M1Dlg.obj
 0001:00010a50       ??_G?$CArray@PAVCString@@PAV1@@@UAEPAXI@Z 00411a50 f M1Dlg.obj
 0001:00010a50       ??_E?$CArray@PAVCString@@PAV1@@@UAEPAXI@Z 00411a50 f M1Dlg.obj
 0001:00010a90       ?SetSize@?$CArray@PAVCString@@PAV1@@@QAEXHH@Z 00411a90 f M1Dlg.obj
 0001:00010dd0       ?ElementAt@?$CArray@PAVCString@@PAV1@@@QAEAAPAVCString@@H@Z 00411dd0 f M1Dlg.obj
 0001:00010e30       ?SetAtGrow@?$CArray@PAVCString@@PAV1@@@QAEXHPAVCString@@@Z 00411e30 f M1Dlg.obj
 0001:00010eb0       ?DestructElements@@YGXPAPAVCString@@H@Z 00411eb0 f M1Dlg.obj
 0001:00010f20       ?SerializeElements@@YGXAAVCArchive@@PAPAVCString@@H@Z 00411f20 f M1Dlg.obj
 0001:00010fb0       ?DumpElements@@YGXAAVCDumpContext@@PBQAVCString@@H@Z 00411fb0 f M1Dlg.obj
 0001:00011000       ?ConstructElements@@YGXPAPAVCString@@H@Z 00412000 f M1Dlg.obj
 0001:000110a0       ??2@YAPAXIPAX@Z            004120a0 f M1Dlg.obj
 0001:000110c0       ?extractlayer2@Mpegtoraw@@QAEXXZ 004120c0 f mpeglayer2.obj
 0001:000128b0       ?_GetBaseMessageMap@CM1App@@KGPBUAFX_MSGMAP@@XZ 004138b0 f M1.obj
 0001:000128c5       ?GetMessageMap@CM1App@@MBEPBUAFX_MSGMAP@@XZ 004138c5 f M1.obj
 0001:000128e0       ??0CM1App@@QAE@XZ          004138e0 f M1.obj
 0001:000129bc       ?InitInstance@CM1App@@UAEHXZ 004139bc f M1.obj
 0001:00012b50       ??_ECM1App@@UAEPAXI@Z      00413b50 f M1.obj
 0001:00012b50       ??_GCM1App@@UAEPAXI@Z      00413b50 f M1.obj
 0001:00012b90       ??1CM1App@@UAE@XZ          00413b90 f M1.obj
 0001:00012bf0       ??1Rawtofile@@UAE@XZ       00413bf0 f rawtofile.obj
 0001:00012c68       ?initialize@Rawtofile@@UAEDPAD@Z 00413c68 f rawtofile.obj
 0001:00012cd0       ?setsoundtype@Rawtofile@@UAEDHHH@Z 00413cd0 f rawtofile.obj
 0001:00012d10       ?putblock@Rawtofile@@UAEDPAXH@Z 00413d10 f rawtofile.obj
 0001:00012d60       ??_GRawtofile@@UAEPAXI@Z   00413d60 f rawtofile.obj
 0001:00012d60       ??_ERawtofile@@UAEPAXI@Z   00413d60 f rawtofile.obj
 0001:00012da0       ?error@Soundplayer@@IAEDH@Z 00413da0 f rawtofile.obj
 0001:00012dd0       ?openfile@Wavefileplayer@@UAEDPAD0@Z 00413dd0 f fileplayer.obj
 0001:000130da       ?playing@Wavefileplayer@@UAEDH@Z 004140da f fileplayer.obj
 0001:00013173       ?openfile@Mpegfileplayer@@UAEDPAD0@Z 00414173 f fileplayer.obj
 0001:0001346b       ?showverbose@Mpegfileplayer@@AAEXXZ 0041446b f fileplayer.obj
 0001:0001350a       ?playing@Mpegfileplayer@@UAEDH@Z 0041450a f fileplayer.obj
 0001:000136a0       ??0Soundinputstreamfromfile@@QAE@H@Z 004146a0 f fileplayer.obj
 0001:000136e0       ??0Soundinputstream@@QAE@XZ 004146e0 f fileplayer.obj
 0001:00013710       ?getblock@Soundinputstreamfromfile@@UAEHPADH@Z 00414710 f fileplayer.obj
 0001:00013760       ?geterrorcode@Soundplayer@@QAEHXZ 00414760 f fileplayer.obj
 0001:00013780       ??0Wavetoraw@@QAE@PAVSoundinputstream@@PAVSoundplayer@@@Z 00414780 f fileplayer.obj
 0001:000137d0       ?error@Fileplayer@@IAEDH@Z 004147d0 f fileplayer.obj
 0001:00013800       ??0Rawplayer@@QAE@XZ       00414800 f fileplayer.obj
 0001:00013870       ??0Soundplayer@@QAE@XZ     00414870 f fileplayer.obj
 0001:000138a0       ??0Rawtofile@@QAE@XZ       004148a0 f fileplayer.obj
 0001:00013910       ?geterrorcode@Wavetoraw@@QAEHXZ 00414910 f fileplayer.obj
 0001:00013930       ??0Soundinputbitstreamfromfile@@QAE@XZ 00414930 f fileplayer.obj
 0001:000139b0       ??0Soundinputbitstream@@QAE@XZ 004149b0 f fileplayer.obj
 0001:000139e0       ??1Soundinputbitstream@@UAE@XZ 004149e0 f fileplayer.obj
 0001:00013a00       ??_GSoundinputbitstream@@UAEPAXI@Z 00414a00 f fileplayer.obj
 0001:00013a00       ??_ESoundinputbitstream@@UAEPAXI@Z 00414a00 f fileplayer.obj
 0001:00013a40       ?geterrorcode@Soundinputbitstreamfromfile@@UAEHXZ 00414a40 f fileplayer.obj
 0001:00013ac0       ?geterrorcode@Bufferinputbitstream@@QAEHXZ 00414ac0 f fileplayer.obj
 0001:00013ae0       ?open@Soundinputbitstreamfromfile@@UAEDPAD@Z 00414ae0 f fileplayer.obj
 0001:00013bf0       ??0Bufferinputbitstream@@QAE@XZ 00414bf0 f fileplayer.obj
 0001:00013c40       ?getbytedirect@Soundinputbitstreamfromfile@@UAEHXZ 00414c40 f fileplayer.obj
 0001:00013c70       ?readbuffer@Soundinputbitstreamfromfile@@UAEDH@Z 00414c70 f fileplayer.obj
 0001:00013ca0       ?getbyte@Soundinputbitstreamfromfile@@UAEHXZ 00414ca0 f fileplayer.obj
 0001:00013cd0       ?getbit@Soundinputbitstreamfromfile@@UAEHXZ 00414cd0 f fileplayer.obj
 0001:00013d00       ?getbit@Bufferinputbitstream@@QAEHXZ 00414d00 f fileplayer.obj
 0001:00013d80       ?getbits@Soundinputbitstreamfromfile@@UAEHH@Z 00414d80 f fileplayer.obj
 0001:00013db0       ?eof@Soundinputbitstreamfromfile@@UAEDXZ 00414db0 f fileplayer.obj
 0001:00013de0       ?eof@Bufferinputbitstream@@QAEDXZ 00414de0 f fileplayer.obj
 0001:00013e10       ?sync@Soundinputbitstreamfromfile@@UAEXXZ 00414e10 f fileplayer.obj
 0001:00013e40       ?sync@Bufferinputbitstream@@QAEXXZ 00414e40 f fileplayer.obj
 0001:00013e60       ??_ESoundinputbitstreamfromfile@@UAEPAXI@Z 00414e60 f fileplayer.obj
 0001:00013e60       ??_GSoundinputbitstreamfromfile@@UAEPAXI@Z 00414e60 f fileplayer.obj
 0001:00013ea0       ??1Soundinputbitstreamfromfile@@UAE@XZ 00414ea0 f fileplayer.obj
 0001:00013f40       ??_GBufferinputbitstream@@QAEPAXI@Z 00414f40 f fileplayer.obj
 0001:00013f80       ??1Bufferinputbitstream@@QAE@XZ 00414f80 f fileplayer.obj
 0001:00013fc0       ??0Mpegtoraw@@QAE@PAVSoundinputbitstream@@PAVSoundplayer@@@Z 00414fc0 f fileplayer.obj
 0001:00014010       ??0Mpegbitwindow@@QAE@XZ   00415010 f fileplayer.obj
 0001:00014040       ?getfrequency@Mpegtoraw@@QAEHXZ 00415040 f fileplayer.obj
 0001:00014070       ?getmode@Mpegtoraw@@QAEHXZ 00415070 f fileplayer.obj
 0001:00014090       ?getbitrate@Mpegtoraw@@QAEHXZ 00415090 f fileplayer.obj
 0001:000140d0       ?getlayer@Mpegtoraw@@QAEHXZ 004150d0 f fileplayer.obj
 0001:000140f0       ?getcrccheck@Mpegtoraw@@QAEDXZ 004150f0 f fileplayer.obj
 0001:00014120       ?geterrorcode@Mpegtoraw@@QAEHXZ 00415120 f fileplayer.obj
 0001:00014140       ?extractlayer1@Mpegtoraw@@QAEXXZ 00415140 f mpeglayer1.obj
 0001:00014670       ?huffmandecoder@Mpegtoraw@@QAEHPBUHUFFMANCODETABLE@@PAH111@Z 00415670 f huffman.obj
 0001:000149b0       ?wgetbit@Mpegtoraw@@QAEHXZ 004159b0 f huffman.obj
 0001:000149e0       ?getbit@Mpegbitwindow@@QAEHXZ 004159e0 f huffman.obj
 0001:00014a40       ??0COptionsDlg@@QAE@PAVCWnd@@@Z 00415a40 f OptionsDlg.obj
 0001:00014af6       ?DoDataExchange@COptionsDlg@@MAEXPAVCDataExchange@@@Z 00415af6 f OptionsDlg.obj
 0001:00014b46       ?_GetBaseMessageMap@COptionsDlg@@KGPBUAFX_MSGMAP@@XZ 00415b46 f OptionsDlg.obj
 0001:00014b5b       ?GetMessageMap@COptionsDlg@@MBEPBUAFX_MSGMAP@@XZ 00415b5b f OptionsDlg.obj
 0001:00014b80       ??_GCOptionsDlg@@UAEPAXI@Z 00415b80 f OptionsDlg.obj
 0001:00014b80       ??_ECOptionsDlg@@UAEPAXI@Z 00415b80 f OptionsDlg.obj
 0001:00014bc0       ??1COptionsDlg@@UAE@XZ     00415bc0 f OptionsDlg.obj
 0001:00014c60       ?getbits@Mpegbitwindow@@QAEHH@Z 00415c60 f bitwindow.obj
 0001:00014d80       ?initialize@Mpegtoraw@@QAEXXZ 00415d80 f mpegtoraw.obj
 0001:00014e43       ?loadheader@Mpegtoraw@@QAEDXZ 00415e43 f mpegtoraw.obj
 0001:00015320       ?run@Mpegtoraw@@QAEDH@Z    00416320 f mpegtoraw.obj
 0001:000154c0       ?error@Mpegtoraw@@QAEDH@Z  004164c0 f mpegtoraw.obj
 0001:000154f0       ?clearrawdata@Mpegtoraw@@QAEXXZ 004164f0 f mpegtoraw.obj
 0001:00015520       ?flushrawdata@Mpegtoraw@@QAEXXZ 00416520 f mpegtoraw.obj
 0001:00015570       ?initialize@Wavetoraw@@QAEDXZ 00416570 f wavetoraw.obj
 0001:000155e0       ?run@Wavetoraw@@QAEDXZ     004165e0 f wavetoraw.obj
 0001:0001573b       ?testwave@Wavetoraw@@AAEDPAD@Z 0041673b f wavetoraw.obj
 0001:00015822       _DirectSoundCreate@12      00416822 f dsound:DSOUND.dll
 0001:00015828       ??3@YAXPAX@Z               00416828 f mfc40d:MFC40D.DLL
 0001:0001582e       ??2@YAPAXI@Z               0041682e f mfc40d:MFC40D.DLL
 0001:00015834       ?SetPos@CSliderCtrl@@QAEXH@Z 00416834 f mfc40d:MFC40D.DLL
 0001:0001583a       ?SetRange@CSliderCtrl@@QAEXHHH@Z 0041683a f mfc40d:MFC40D.DLL
 0001:00015840       ?GetPos@CSliderCtrl@@QBEHXZ 00416840 f mfc40d:MFC40D.DLL
 0001:00015846       ?PreInitDialog@CDialog@@MAEXXZ 00416846 f mfc40d:MFC40D.DLL
 0001:0001584c       ?OnCancel@CDialog@@MAEXXZ  0041684c f mfc40d:MFC40D.DLL
 0001:00015852       ?OnOK@CDialog@@MAEXXZ      00416852 f mfc40d:MFC40D.DLL
 0001:00015858       ?OnSetFont@CDialog@@UAEXPAVCFont@@@Z 00416858 f mfc40d:MFC40D.DLL
 0001:0001585e       ?OnInitDialog@CDialog@@UAEHXZ 0041685e f mfc40d:MFC40D.DLL
 0001:00015864       ?DoModal@CDialog@@UAEHXZ   00416864 f mfc40d:MFC40D.DLL
 0001:0001586a       ?SetOccDialogInfo@CDialog@@MAEHPAU_AFX_OCC_DIALOG_INFO@@@Z 0041686a f mfc40d:MFC40D.DLL
 0001:00015870       ?IsFrameWnd@CWnd@@UBEHXZ   00416870 f mfc40d:MFC40D.DLL
 0001:00015876       ?CheckAutoCenter@CDialog@@UAEHXZ 00416876 f mfc40d:MFC40D.DLL
 0001:0001587c       ?OnChildNotify@CWnd@@MAEHIIJPAJ@Z 0041687c f mfc40d:MFC40D.DLL
 0001:00015882       ?PostNcDestroy@CWnd@@MAEXXZ 00416882 f mfc40d:MFC40D.DLL
 0001:00015888       ?DefWindowProcA@CWnd@@MAEJIIJ@Z 00416888 f mfc40d:MFC40D.DLL
 0001:0001588e       ?OnWndMsg@CWnd@@MAEHIIJPAJ@Z 0041688e f mfc40d:MFC40D.DLL
 0001:00015894       ?WindowProc@CWnd@@MAEJIIJ@Z 00416894 f mfc40d:MFC40D.DLL
 0001:0001589a       ?OnAmbientProperty@CWnd@@UAEHPAVCOleControlSite@@JPAUtagVARIANT@@@Z 0041689a f mfc40d:MFC40D.DLL
 0001:000158a0       ?PreTranslateMessage@CDialog@@UAEHPAUtagMSG@@@Z 004168a0 f mfc40d:MFC40D.DLL
 0001:000158a6       ?EndModalState@CWnd@@UAEXXZ 004168a6 f mfc40d:MFC40D.DLL
 0001:000158ac       ?BeginModalState@CWnd@@UAEXXZ 004168ac f mfc40d:MFC40D.DLL
 0001:000158b2       ?GetSuperWndProcAddr@CWnd@@MAEPAP6GJPAUHWND__@@IIJ@ZXZ 004168b2 f mfc40d:MFC40D.DLL
 0001:000158b8       ?OnNotify@CWnd@@MAEHIJPAJ@Z 004168b8 f mfc40d:MFC40D.DLL
 0001:000158be       ?OnCommand@CWnd@@MAEHIJ@Z  004168be f mfc40d:MFC40D.DLL
 0001:000158c4       ?EndModalLoop@CWnd@@UAEXH@Z 004168c4 f mfc40d:MFC40D.DLL
 0001:000158ca       ?ContinueModal@CWnd@@UAEHXZ 004168ca f mfc40d:MFC40D.DLL
 0001:000158d0       ?WinHelpA@CWnd@@UAEXKI@Z   004168d0 f mfc40d:MFC40D.DLL
 0001:000158d6       ?GetScrollBarCtrl@CWnd@@UBEPAVCScrollBar@@H@Z 004168d6 f mfc40d:MFC40D.DLL
 0001:000158dc       ?OnToolHitTest@CWnd@@UBEHVCPoint@@PAUtagTOOLINFOA@@@Z 004168dc f mfc40d:MFC40D.DLL
 0001:000158e2       ?CalcWindowRect@CWnd@@UAEXPAUtagRECT@@I@Z 004168e2 f mfc40d:MFC40D.DLL
 0001:000158e8       ?PreCreateWindow@CWnd@@UAEHAAUtagCREATESTRUCTA@@@Z 004168e8 f mfc40d:MFC40D.DLL
 0001:000158ee       ?DestroyWindow@CWnd@@UAEHXZ 004168ee f mfc40d:MFC40D.DLL
 0001:000158f4       ?Create@CWnd@@UAEHPBD0KABUtagRECT@@PAV1@IPAUCCreateContext@@@Z 004168f4 f mfc40d:MFC40D.DLL
 0001:000158fa       ?PreSubclassWindow@CWnd@@UAEXXZ 004168fa f mfc40d:MFC40D.DLL
 0001:00015900       ?GetConnectionHook@CCmdTarget@@MAEPAUIConnectionPoint@@ABU_GUID@@@Z 00416900 f mfc40d:MFC40D.DLL
 0001:00015906       ?GetExtraConnectionPoints@CCmdTarget@@MAEHPAVCPtrArray@@@Z 00416906 f mfc40d:MFC40D.DLL
 0001:0001590c       ?GetInterfaceHook@CCmdTarget@@UAEPAUIUnknown@@PBX@Z 0041690c f mfc40d:MFC40D.DLL
 0001:00015912       ?OnCreateAggregates@CCmdTarget@@UAEHXZ 00416912 f mfc40d:MFC40D.DLL
 0001:00015918       ?GetEventSinkMap@CCmdTarget@@MBEPBUAFX_EVENTSINKMAP@@XZ 00416918 f mfc40d:MFC40D.DLL
 0001:0001591e       ?GetInterfaceMap@CCmdTarget@@MBEPBUAFX_INTERFACEMAP@@XZ 0041691e f mfc40d:MFC40D.DLL
 0001:00015924       ?GetConnectionMap@CCmdTarget@@MBEPBUAFX_CONNECTIONMAP@@XZ 00416924 f mfc40d:MFC40D.DLL
 0001:0001592a       ?GetDispatchMap@CCmdTarget@@MBEPBUAFX_DISPMAP@@XZ 0041692a f mfc40d:MFC40D.DLL
 0001:00015930       ?GetTypeLib@CCmdTarget@@UAEJKPAPAUITypeLib@@@Z 00416930 f mfc40d:MFC40D.DLL
 0001:00015936       ?GetTypeLibCache@CCmdTarget@@UAEPAVCTypeLibCache@@XZ 00416936 f mfc40d:MFC40D.DLL
 0001:0001593c       ?GetTypeInfoCount@CCmdTarget@@UAEIXZ 0041693c f mfc40d:MFC40D.DLL
 0001:00015942       ?GetDispatchIID@CCmdTarget@@UAEHPAU_GUID@@@Z 00416942 f mfc40d:MFC40D.DLL
 0001:00015948       ?IsInvokeAllowed@CCmdTarget@@UAEHJ@Z 00416948 f mfc40d:MFC40D.DLL
 0001:0001594e       ?OnFinalRelease@CWnd@@UAEXXZ 0041694e f mfc40d:MFC40D.DLL
 0001:00015954       ?OnCmdMsg@CDialog@@UAEHIHPAXPAUAFX_CMDHANDLERINFO@@@Z 00416954 f mfc40d:MFC40D.DLL
 0001:0001595a       ?Dump@CDialog@@UBEXAAVCDumpContext@@@Z 0041695a f mfc40d:MFC40D.DLL
 0001:00015960       ?AssertValid@CDialog@@UBEXXZ 00416960 f mfc40d:MFC40D.DLL
 0001:00015966       ?Serialize@CObject@@UAEXAAVCArchive@@@Z 00416966 f mfc40d:MFC40D.DLL
 0001:0001596c       ?GetRuntimeClass@CDialog@@UBEPAUCRuntimeClass@@XZ 0041696c f mfc40d:MFC40D.DLL
 0001:00015972       ??1CDialog@@UAE@XZ         00416972 f mfc40d:MFC40D.DLL
 0001:00015978       ??0CDialog@@QAE@IPAVCWnd@@@Z 00416978 f mfc40d:MFC40D.DLL
 0001:0001597e       ??3CObject@@SGXPAX@Z       0041697e f mfc40d:MFC40D.DLL
 0001:00015984       ?DoDataExchange@CWnd@@MAEXPAVCDataExchange@@@Z 00416984 f mfc40d:MFC40D.DLL
 0001:0001598a       ?messageMap@CDialog@@1UAFX_MSGMAP@@B 0041698a f mfc40d:MFC40D.DLL
 0001:00015990       ?OnContextMenu@CWnd@@IAEXPAV1@VCPoint@@@Z 00416990 f mfc40d:MFC40D.DLL
 0001:00015996       ?SetIcon@CButton@@QAEPAUHICON__@@PAU2@@Z 00416996 f mfc40d:MFC40D.DLL
 0001:0001599c       ?SetWindowTextA@CWnd@@QAEXPBD@Z 0041699c f mfc40d:MFC40D.DLL
 0001:000159a2       ?KillTimer@CWnd@@QAEHH@Z   004169a2 f mfc40d:MFC40D.DLL
 0001:000159a8       ?SetTimer@CWnd@@QAEIIIP6GXPAUHWND__@@IIK@Z@Z 004169a8 f mfc40d:MFC40D.DLL
 0001:000159ae       ?GetBuffer@CString@@QAEPADH@Z 004169ae f mfc40d:MFC40D.DLL
 0001:000159b4       ??0CString@@QAE@PBD@Z      004169b4 f mfc40d:MFC40D.DLL
 0001:000159ba       ??0CStdioFile@@QAE@PBDI@Z  004169ba f mfc40d:MFC40D.DLL
 0001:000159c0       ??2CObject@@SGPAXI@Z       004169c0 f mfc40d:MFC40D.DLL
 0001:000159c6       ??0CFont@@QAE@XZ           004169c6 f mfc40d:MFC40D.DLL
 0001:000159cc       ??1CFont@@UAE@XZ           004169cc f mfc40d:MFC40D.DLL
 0001:000159d2       ??1CStatic@@UAE@XZ         004169d2 f mfc40d:MFC40D.DLL
 0001:000159d8       ??1CButton@@UAE@XZ         004169d8 f mfc40d:MFC40D.DLL
 0001:000159de       ?LoadIconA@CWinApp@@QBEPAUHICON__@@I@Z 004169de f mfc40d:MFC40D.DLL
 0001:000159e4       ?AfxGetApp@@YGPAVCWinApp@@XZ 004169e4 f mfc40d:MFC40D.DLL
 0001:000159ea       ??0CButton@@QAE@XZ         004169ea f mfc40d:MFC40D.DLL
 0001:000159f0       ??0CStatic@@QAE@XZ         004169f0 f mfc40d:MFC40D.DLL
 0001:000159f6       ?DDX_Control@@YGXPAVCDataExchange@@HAAVCWnd@@@Z 004169f6 f mfc40d:MFC40D.DLL
 0001:000159fc       ??1CString@@QAE@XZ         004169fc f mfc40d:MFC40D.DLL
 0001:00015a02       ?SetFont@CWnd@@QAEXPAVCFont@@H@Z 00416a02 f mfc40d:MFC40D.DLL
 0001:00015a08       ?CreatePointFont@CFont@@QAEHHPBDPAVCDC@@@Z 00416a08 f mfc40d:MFC40D.DLL
 0001:00015a0e       ?DragAcceptFiles@CWnd@@QAEXH@Z 00416a0e f mfc40d:MFC40D.DLL
 0001:00015a14       ?GetSafeHwnd@CWnd@@QBEPAUHWND__@@XZ 00416a14 f mfc40d:MFC40D.DLL
 0001:00015a1a       ?Create@CDialog@@QAEHIPAVCWnd@@@Z 00416a1a f mfc40d:MFC40D.DLL
 0001:00015a20       ??2CObject@@SGPAXIPBDH@Z   00416a20 f mfc40d:MFC40D.DLL
 0001:00015a26       ?SetIcon@CWnd@@QAEPAUHICON__@@PAU2@H@Z 00416a26 f mfc40d:MFC40D.DLL
 0001:00015a2c       ?AppendMenuA@CMenu@@QAEHIIPBD@Z 00416a2c f mfc40d:MFC40D.DLL
 0001:00015a32       ??BCString@@QBEPBDXZ       00416a32 f mfc40d:MFC40D.DLL
 0001:00015a38       ?IsEmpty@CString@@QBEHXZ   00416a38 f mfc40d:MFC40D.DLL
 0001:00015a3e       ?LoadStringA@CString@@QAEHI@Z 00416a3e f mfc40d:MFC40D.DLL
 0001:00015a44       ??0CString@@QAE@XZ         00416a44 f mfc40d:MFC40D.DLL
 0001:00015a4a       ?GetSystemMenu@CWnd@@QBEPAVCMenu@@H@Z 00416a4a f mfc40d:MFC40D.DLL
 0001:00015a50       ?OnSysCommand@CWnd@@IAEXIJ@Z 00416a50 f mfc40d:MFC40D.DLL
 0001:00015a56       ??1CPaintDC@@UAE@XZ        00416a56 f mfc40d:MFC40D.DLL
 0001:00015a5c       ?OnPaint@CWnd@@IAEXXZ      00416a5c f mfc40d:MFC40D.DLL
 0001:00015a62       ?DrawIcon@CDC@@QAEHHHPAUHICON__@@@Z 00416a62 f mfc40d:MFC40D.DLL
 0001:00015a68       ?Height@CRect@@QBEHXZ      00416a68 f mfc40d:MFC40D.DLL
 0001:00015a6e       ?Width@CRect@@QBEHXZ       00416a6e f mfc40d:MFC40D.DLL
 0001:00015a74       ?GetClientRect@CWnd@@QBEXPAUtagRECT@@@Z 00416a74 f mfc40d:MFC40D.DLL
 0001:00015a7a       ??0CRect@@QAE@XZ           00416a7a f mfc40d:MFC40D.DLL
 0001:00015a80       ?SendMessageA@CWnd@@QAEJIIJ@Z 00416a80 f mfc40d:MFC40D.DLL
 0001:00015a86       ?GetSafeHdc@CDC@@QBEPAUHDC__@@XZ 00416a86 f mfc40d:MFC40D.DLL
 0001:00015a8c       ??0CPaintDC@@QAE@PAVCWnd@@@Z 00416a8c f mfc40d:MFC40D.DLL
 0001:00015a92       ?IsIconic@CWnd@@QBEHXZ     00416a92 f mfc40d:MFC40D.DLL
 0001:00015a98       ?GetCheck@CButton@@QBEHXZ  00416a98 f mfc40d:MFC40D.DLL
 0001:00015a9e       ?SetFocus@CWnd@@QAEPAV1@XZ 00416a9e f mfc40d:MFC40D.DLL
 0001:00015aa4       ?SetForegroundWindow@CWnd@@QAEHXZ 00416aa4 f mfc40d:MFC40D.DLL
 0001:00015aaa       ??2@YAPAXIPBDH@Z           00416aaa f mfc40d:MFC40D.DLL
 0001:00015ab0       ?SetWindowPos@CWnd@@QAEHPBV1@HHHHI@Z 00416ab0 f mfc40d:MFC40D.DLL
 0001:00015ab6       ?GetWindowPlacement@CWnd@@QBEHPAUtagWINDOWPLACEMENT@@@Z 00416ab6 f mfc40d:MFC40D.DLL
 0001:00015abc       ?ShowWindow@CWnd@@QAEHH@Z  00416abc f mfc40d:MFC40D.DLL
 0001:00015ac2       ?GetRuntimeClass@CObject@@UBEPAUCRuntimeClass@@XZ 00416ac2 f mfc40d:MFC40D.DLL
 0001:00015ac8       ??1CObject@@UAE@XZ         00416ac8 f mfc40d:MFC40D.DLL
 0001:00015ace       ??0CObject@@IAE@XZ         00416ace f mfc40d:MFC40D.DLL
 0001:00015ad4       ?AfxAssertValidObject@@YGXPBVCObject@@PBDH@Z 00416ad4 f mfc40d:MFC40D.DLL
 0001:00015ada       ?ReadCount@CArchive@@QAEKXZ 00416ada f mfc40d:MFC40D.DLL
 0001:00015ae0       ?WriteCount@CArchive@@QAEXK@Z 00416ae0 f mfc40d:MFC40D.DLL
 0001:00015ae6       ?IsStoring@CArchive@@QBEHXZ 00416ae6 f mfc40d:MFC40D.DLL
 0001:00015aec       ??6CDumpContext@@QAEAAV0@PBD@Z 00416aec f mfc40d:MFC40D.DLL
 0001:00015af2       ?GetDepth@CDumpContext@@QBEHXZ 00416af2 f mfc40d:MFC40D.DLL
 0001:00015af8       ??6CDumpContext@@QAEAAV0@H@Z 00416af8 f mfc40d:MFC40D.DLL
 0001:00015afe       ?Dump@CObject@@UBEXAAVCDumpContext@@@Z 00416afe f mfc40d:MFC40D.DLL
 0001:00015b04       ?AfxAssertFailedLine@@YGHPBDH@Z 00416b04 f mfc40d:MFC40D.DLL
 0001:00015b0a       ?AfxIsValidAddress@@YGHPBXIH@Z 00416b0a f mfc40d:MFC40D.DLL
 0001:00015b10       ?AssertValid@CObject@@UBEXXZ 00416b10 f mfc40d:MFC40D.DLL
 0001:00015b16       ?Read@CArchive@@QAEIPAXI@Z 00416b16 f mfc40d:MFC40D.DLL
 0001:00015b1c       ?Write@CArchive@@QAEXPBXI@Z 00416b1c f mfc40d:MFC40D.DLL
 0001:00015b22       ?OnHelp@CWinApp@@IAEXXZ    00416b22 f mfc40d:MFC40D.DLL
 0001:00015b28       ?messageMap@CWinApp@@1UAFX_MSGMAP@@B 00416b28 f mfc40d:MFC40D.DLL
 0001:00015b2e       ?WinHelpA@CWinApp@@UAEXKI@Z 00416b2e f mfc40d:MFC40D.DLL
 0001:00015b34       ?OnDDECommand@CWinApp@@UAEHPAD@Z 00416b34 f mfc40d:MFC40D.DLL
 0001:00015b3a       ?DoWaitCursor@CWinApp@@UAEXH@Z 00416b3a f mfc40d:MFC40D.DLL
 0001:00015b40       ?DoMessageBox@CWinApp@@UAEHPBDII@Z 00416b40 f mfc40d:MFC40D.DLL
 0001:00015b46       ?SaveAllModified@CWinApp@@UAEHXZ 00416b46 f mfc40d:MFC40D.DLL
 0001:00015b4c       ?InitApplication@CWinApp@@UAEHXZ 00416b4c f mfc40d:MFC40D.DLL
 0001:00015b52       ?AddToRecentFileList@CWinApp@@UAEXPBD@Z 00416b52 f mfc40d:MFC40D.DLL
 0001:00015b58       ?OpenDocumentFile@CWinApp@@UAEPAVCDocument@@PBD@Z 00416b58 f mfc40d:MFC40D.DLL
 0001:00015b5e       ?Delete@CWinThread@@UAEXXZ 00416b5e f mfc40d:MFC40D.DLL
 0001:00015b64       ?GetMainWnd@CWinThread@@UAEPAVCWnd@@XZ 00416b64 f mfc40d:MFC40D.DLL
 0001:00015b6a       ?ProcessMessageFilter@CWinThread@@UAEHHPAUtagMSG@@@Z 00416b6a f mfc40d:MFC40D.DLL
 0001:00015b70       ?ProcessWndProcException@CWinApp@@UAEJPAVCException@@PBUtagMSG@@@Z 00416b70 f mfc40d:MFC40D.DLL
 0001:00015b76       ?ExitInstance@CWinApp@@UAEHXZ 00416b76 f mfc40d:MFC40D.DLL
 0001:00015b7c       ?IsIdleMessage@CWinThread@@UAEHPAUtagMSG@@@Z 00416b7c f mfc40d:MFC40D.DLL
 0001:00015b82       ?OnIdle@CWinApp@@UAEHJ@Z   00416b82 f mfc40d:MFC40D.DLL
 0001:00015b88       ?PumpMessage@CWinThread@@UAEHXZ 00416b88 f mfc40d:MFC40D.DLL
 0001:00015b8e       ?PreTranslateMessage@CWinThread@@UAEHPAUtagMSG@@@Z 00416b8e f mfc40d:MFC40D.DLL
 0001:00015b94       ?Run@CWinApp@@UAEHXZ       00416b94 f mfc40d:MFC40D.DLL
 0001:00015b9a       ?OnFinalRelease@CCmdTarget@@UAEXXZ 00416b9a f mfc40d:MFC40D.DLL
 0001:00015ba0       ?OnCmdMsg@CCmdTarget@@UAEHIHPAXPAUAFX_CMDHANDLERINFO@@@Z 00416ba0 f mfc40d:MFC40D.DLL
 0001:00015ba6       ?Dump@CWinApp@@UBEXAAVCDumpContext@@@Z 00416ba6 f mfc40d:MFC40D.DLL
 0001:00015bac       ?AssertValid@CWinApp@@UBEXXZ 00416bac f mfc40d:MFC40D.DLL
 0001:00015bb2       ?GetRuntimeClass@CWinApp@@UBEPAUCRuntimeClass@@XZ 00416bb2 f mfc40d:MFC40D.DLL
 0001:00015bb8       ??1CWinApp@@UAE@XZ         00416bb8 f mfc40d:MFC40D.DLL
 0001:00015bbe       ??0CWinApp@@QAE@PBD@Z      00416bbe f mfc40d:MFC40D.DLL
 0001:00015bc4       ?Enable3dControls@CWinApp@@IAEHXZ 00416bc4 f mfc40d:MFC40D.DLL
 0001:00015bca       ?SetDialogBkColor@CWinApp@@IAEXKK@Z 00416bca f mfc40d:MFC40D.DLL
 0001:00015bd0       ??1CSliderCtrl@@UAE@XZ     00416bd0 f mfc40d:MFC40D.DLL
 0001:00015bd6       ??0CSliderCtrl@@QAE@XZ     00416bd6 f mfc40d:MFC40D.DLL
 0001:00015bdc       _fopen                     00416bdc f msvcrtd:MSVCR40D.dll
 0001:00015be2       ___p__iob                  00416be2 f msvcrtd:MSVCR40D.dll
 0001:00015be8       _fclose                    00416be8 f msvcrtd:MSVCR40D.dll
 0001:00015bee       _getc                      00416bee f msvcrtd:MSVCR40D.dll
 0001:00015bf4       _fread                     00416bf4 f msvcrtd:MSVCR40D.dll
 0001:00015bfa       ___CxxFrameHandler         00416bfa f msvcrtd:MSVCR40D.dll
 0001:00015c00       __purecall                 00416c00 f msvcrtd:MSVCR40D.dll
 0001:00015c06       __adj_fdivr_m64            00416c06 f msvcrtd:MSVCR40D.dll
 0001:00015c0c       _cos                       00416c0c f msvcrtd:MSVCR40D.dll
 0001:00015c12       __adj_fdiv_m64             00416c12 f msvcrtd:MSVCR40D.dll
 0001:00015c18       __ftol                     00416c18 f msvcrtd:MSVCR40D.dll
 0001:00015c1e       _sin                       00416c1e f msvcrtd:MSVCR40D.dll
 0001:00015c24       __adj_fdivr_m32            00416c24 f msvcrtd:MSVCR40D.dll
 0001:00015c2a       _sqrt                      00416c2a f msvcrtd:MSVCR40D.dll
 0001:00015c30       _pow                       00416c30 f msvcrtd:MSVCR40D.dll
 0001:00015c36       _memcpy                    00416c36 f msvcrtd:MSVCR40D.dll
 0001:00015c40       __chkstk                   00416c40   msvcrtd:chkstk.obj
 0001:00015c40       __alloca_probe             00416c40   msvcrtd:chkstk.obj
 0001:00015c70       _putc                      00416c70 f msvcrtd:MSVCR40D.dll
 0001:00015c76       _memset                    00416c76 f msvcrtd:MSVCR40D.dll
 0001:00015c7c       _log                       00416c7c f msvcrtd:MSVCR40D.dll
 0001:00015c82       _strcpy                    00416c82 f msvcrtd:MSVCR40D.dll
 0001:00015c88       __itoa                     00416c88 f msvcrtd:MSVCR40D.dll
 0001:00015c8e       _abs                       00416c8e f msvcrtd:MSVCR40D.dll
 0001:00015c94       _strrchr                   00416c94 f msvcrtd:MSVCR40D.dll
 0001:00015c9a       _strlen                    00416c9a f msvcrtd:MSVCR40D.dll
 0001:00015ca0       _strstr                    00416ca0 f msvcrtd:MSVCR40D.dll
 0001:00015ca6       _fprintf                   00416ca6 f msvcrtd:MSVCR40D.dll
 0001:00015cb0       __onexit                   00416cb0 f msvcrtd:atonexit.obj
 0001:00015d80       _atexit                    00416d80 f msvcrtd:atonexit.obj
 0001:00015db0       _malloc                    00416db0 f msvcrtd:MSVCR40D.dll
 0001:00015dc0       _WinMainCRTStartup         00416dc0 f msvcrtd:crtexew.obj
 0001:00015ffe       ___dllonexit               00416ffe f msvcrtd:MSVCR40D.dll
 0001:00016004       __exit                     00417004 f msvcrtd:MSVCR40D.dll
 0001:0001600a       __XcptFilter               0041700a f msvcrtd:MSVCR40D.dll
 0001:00016010       _exit                      00417010 f msvcrtd:MSVCR40D.dll
 0001:00016016       ___p__acmdln               00417016 f msvcrtd:MSVCR40D.dll
 0001:0001601c       __initterm                 0041701c f msvcrtd:MSVCR40D.dll
 0001:00016022       ___getmainargs             00417022 f msvcrtd:MSVCR40D.dll
 0001:00016030       __setdefaultprecision      00417030 f msvcrtd:fp8.obj
 0001:0001604e       ___setusermatherr          0041704e f msvcrtd:MSVCR40D.dll
 0001:00016060       __matherr                  00417060 f msvcrtd:merr.obj
 0001:00016080       __setargv                  00417080 f msvcrtd:dllargv.obj
 0001:0001608c       ___p__commode              0041708c f msvcrtd:MSVCR40D.dll
 0001:00016092       ___p__fmode                00417092 f msvcrtd:MSVCR40D.dll
 0001:00016098       ___set_app_type            00417098 f msvcrtd:MSVCR40D.dll
 0001:0001609e       __except_handler3          0041709e f msvcrtd:MSVCR40D.dll
 0001:000160a4       __controlfp                004170a4 f msvcrtd:MSVCR40D.dll
 0001:000160aa       _Sleep@4                   004170aa f kernel32:KERNEL32.dll
 0001:000160b0       _SetThreadPriority@8       004170b0 f kernel32:KERNEL32.dll
 0001:000160b6       _CreateThread@24           004170b6 f kernel32:KERNEL32.dll
 0001:000160bc       _GetExitCodeThread@8       004170bc f kernel32:KERNEL32.dll
 0001:000160c2       _GetVersion@0              004170c2 f kernel32:KERNEL32.dll
 0001:000160c8       _GetModuleHandleA@4        004170c8 f kernel32:KERNEL32.dll
 0001:000160ce       _GetStartupInfoA@4         004170ce f kernel32:KERNEL32.dll
 0001:000160d4       _MessageBoxA@16            004170d4 f user32:USER32.dll
 0001:000160da       _GetSystemMetrics@4        004170da f user32:USER32.dll
 0001:000160e0       _DragQueryFileA@16         004170e0 f shell32:SHELL32.dll
 0001:000160f0       _WinMain@16                004170f0 f mfcs40d:appmodul.obj
 0001:00016120       ?AfxInitialize@@YGHHK@Z    00417120 f mfcs40d:appmodul.obj
 0001:00016190       ??0_AFX_TERM_APP_STATE@@QAE@XZ 00417190 f mfcs40d:appmodul.obj
 0001:000161fa       __close                    004171fa f msvcrtd:MSVCR40D.dll
 0001:00016200       __write                    00417200 f msvcrtd:MSVCR40D.dll
 0001:00016206       __open                     00417206 f msvcrtd:MSVCR40D.dll
 0001:0001620c       __read                     0041720c f msvcrtd:MSVCR40D.dll
 0001:00016212       __setmbcp                  00417212 f msvcrtd:MSVCR40D.dll
 0001:00016218       ?AfxWinMain@@YGHPAUHINSTANCE__@@0PADH@Z 00417218 f mfc40d:MFC40D.DLL
 0001:0001621e       ?AfxGetModuleState@@YGPAVAFX_MODULE_STATE@@XZ 0041721e f mfc40d:MFC40D.DLL
 0002:00000058       ??_7Rawplayer@@6B@         00418058   rawplayer.obj
 0002:00000070       ??_7Soundplayer@@6B@       00418070   rawplayer.obj
 0002:000002b0       ?messageMap@CPlaylistDlg@@1UAFX_MSGMAP@@B 004182b0   PlaylistDlg.obj
 0002:000002b8       ?_messageEntries@CPlaylistDlg@@0PBUAFX_MSGMAP_ENTRY@@B 004182b8   PlaylistDlg.obj
 0002:000002d0       ??_7CPlaylistDlg@@6B@      004182d0   PlaylistDlg.obj
 0002:000003a8       ?messageMap@CAboutDlg@@1UAFX_MSGMAP@@B 004183a8   M1Dlg.obj
 0002:000003b0       ?_messageEntries@CAboutDlg@@0PBUAFX_MSGMAP_ENTRY@@B 004183b0   M1Dlg.obj
 0002:000003c8       ?messageMap@CM1Dlg@@1UAFX_MSGMAP@@B 004183c8   M1Dlg.obj
 0002:000003d0       ?_messageEntries@CM1Dlg@@0PBUAFX_MSGMAP_ENTRY@@B 004183d0   M1Dlg.obj
 0002:000004f0       ??_7Mpegfileplayer@@6B@    004184f0   M1Dlg.obj
 0002:00000500       ??_7Fileplayer@@6B@        00418500   M1Dlg.obj
 0002:00000510       ??_7CAboutDlg@@6B@         00418510   M1Dlg.obj
 0002:000005e8       ??_7CM1Dlg@@6B@            004185e8   M1Dlg.obj
 0002:000006c0       ??_7?$CArray@PAVCString@@PAV1@@@6B@ 004186c0   M1Dlg.obj
 0002:000006e8       ?messageMap@CM1App@@1UAFX_MSGMAP@@B 004186e8   M1.obj
 0002:000006f0       ?_messageEntries@CM1App@@0PBUAFX_MSGMAP_ENTRY@@B 004186f0   M1.obj
 0002:00000720       ??_7CM1App@@6B@            00418720   M1.obj
 0002:000007c0       ??_7Rawtofile@@6B@         004187c0   rawtofile.obj
 0002:000007d4       ??_7Soundinputstreamfromfile@@6B@ 004187d4   fileplayer.obj
 0002:000007d8       ??_7Soundinputstream@@6B@  004187d8   fileplayer.obj
 0002:000007e0       ??_7Soundinputbitstreamfromfile@@6B@ 004187e0   fileplayer.obj
 0002:00000808       ??_7Soundinputbitstream@@6B@ 00418808   fileplayer.obj
 0002:00000838       ?messageMap@COptionsDlg@@1UAFX_MSGMAP@@B 00418838   OptionsDlg.obj
 0002:00000840       ?_messageEntries@COptionsDlg@@0PBUAFX_MSGMAP_ENTRY@@B 00418840   OptionsDlg.obj
 0002:00000858       ??_7COptionsDlg@@6B@       00418858   OptionsDlg.obj
 0002:00001f40       ?ht@Mpegtoraw@@2PBUHUFFMANCODETABLE@@B 00419f40   huffmantable.obj
 0002:00002278       ?frequencies@Mpegtoraw@@2PBHB 0041a278   mpegtable.obj
 0002:00002288       ?bitrate@Mpegtoraw@@2PAY0P@HA 0041a288   mpegtable.obj
 0002:00002340       ?scalefactorstable@Mpegtoraw@@2PBMB 0041a340   mpegtable.obj
 0002:00002440       ?factortable@Mpegtoraw@@2PBMB 0041a440   mpegtable.obj
 0002:00002480       ?offsettable@Mpegtoraw@@2PBMB 0041a480   mpegtable.obj
 0002:000024c0       ?bitalloclengthtable@Mpegtoraw@@2PAY0CA@HA 0041a4c0   mpegtable.obj
 0002:000025c0       ?group5bits@Mpegtoraw@@2PBMB 0041a5c0   mpegtable.obj
 0002:00002708       ?group7bits@Mpegtoraw@@2PBMB 0041a708   mpegtable.obj
 0002:00002ce8       ?group10bits@Mpegtoraw@@2PBMB 0041ace8   mpegtable.obj
 0002:00004f18       ?codelengthtableA@Mpegtoraw@@2PBHB 0041cf18   mpegtable.obj
 0002:00004f58       ?codelengthtableB1@Mpegtoraw@@2PBHB 0041cf58   mpegtable.obj
 0002:00004f98       ?codelengthtableB2@Mpegtoraw@@2PBHB 0041cf98   mpegtable.obj
 0002:00004fd8       ?codelengthtableB3@Mpegtoraw@@2PBHB 0041cfd8   mpegtable.obj
 0002:00004ff8       ?codelengthtableB4@Mpegtoraw@@2PBHB 0041cff8   mpegtable.obj
 0002:00005008       ?factortableA@Mpegtoraw@@2PBMB 0041d008   mpegtable.obj
 0002:00005048       ?factortableB1@Mpegtoraw@@2PBMB 0041d048   mpegtable.obj
 0002:00005088       ?factortableB2@Mpegtoraw@@2PBMB 0041d088   mpegtable.obj
 0002:000050c8       ?factortableB3@Mpegtoraw@@2PBMB 0041d0c8   mpegtable.obj
 0002:000050e8       ?factortableB4@Mpegtoraw@@2PBMB 0041d0e8   mpegtable.obj
 0002:000050f8       ?ctableA@Mpegtoraw@@2PBMB  0041d0f8   mpegtable.obj
 0002:00005138       ?ctableB1@Mpegtoraw@@2PBMB 0041d138   mpegtable.obj
 0002:00005178       ?ctableB2@Mpegtoraw@@2PBMB 0041d178   mpegtable.obj
 0002:000051b8       ?ctableB3@Mpegtoraw@@2PBMB 0041d1b8   mpegtable.obj
 0002:000051d8       ?ctableB4@Mpegtoraw@@2PBMB 0041d1d8   mpegtable.obj
 0002:000051e8       ?dtableA@Mpegtoraw@@2PBMB  0041d1e8   mpegtable.obj
 0002:00005228       ?dtableB1@Mpegtoraw@@2PBMB 0041d228   mpegtable.obj
 0002:00005268       ?dtableB2@Mpegtoraw@@2PBMB 0041d268   mpegtable.obj
 0002:000052a8       ?dtableB3@Mpegtoraw@@2PBMB 0041d2a8   mpegtable.obj
 0002:000052c8       ?dtableB4@Mpegtoraw@@2PBMB 0041d2c8   mpegtable.obj
 0002:000052d8       ?filter@Mpegtoraw@@2PBMB   0041d2d8   mpegtable.obj
 0003:00000000       ___xc_a                    0041f000   msvcrtd:cinitexe.obj
 0003:0000008c       ___xc_z                    0041f08c   msvcrtd:cinitexe.obj
 0003:00000090       ___xi_a                    0041f090   msvcrtd:cinitexe.obj
 0003:00000094       ___xi_z                    0041f094   msvcrtd:cinitexe.obj
 0003:00000884       ?counter@@3JA              0041f884   M1Dlg.obj
 0003:000008c8       ?stop@@3DA                 0041f8c8   M1Dlg.obj
 0003:000008cc       ?playlistsong@@3HA         0041f8cc   M1Dlg.obj
 0003:00000ab8       ??_C@_01BJG@?6?$AA@        0041fab8   M1Dlg.obj
 0003:00000abc       ??_C@_09LOPF@?5elements?$AA@ 0041fabc   M1Dlg.obj
 0003:00000ac8       ??_C@_05KIFI@with?5?$AA@   0041fac8   M1Dlg.obj
 0003:00000b90       ?modestring@Mpegtoraw@@2PAPBDA 0041fb90   mpegtable.obj
 0003:00000ba0       ?grouptableA@Mpegtoraw@@2PAPBMA 0041fba0   mpegtable.obj
 0003:00000be0       ?grouptableB1@Mpegtoraw@@2PAPBMA 0041fbe0   mpegtable.obj
 0003:00000c20       ?grouptableB234@Mpegtoraw@@2PAPBMA 0041fc20   mpegtable.obj
 0003:00000c90       ___win32sflag              0041fc90   msvcrtd:atonexit.obj
 0003:00000c98       __dowildcard               0041fc98   msvcrtd:wildcard.obj
 0003:00000c9c       __newmode                  0041fc9c   msvcrtd:_newmode.obj
 0003:00000ca0       ___defaultmatherr          0041fca0   msvcrtd:merr.obj
 0003:00000ca4       __commode                  0041fca4   msvcrtd:xncommod.obj
 0003:00000ca8       __fmode                    0041fca8   msvcrtd:xtxtmode.obj
 0003:00011980       ?usePlayList@@3HA          00430980   M1Dlg.obj
 0003:00011984       ?bitrate@@3JA              00430984   M1Dlg.obj
 0003:00011988       ?d@@3PAVCM1Dlg@@A          00430988   M1Dlg.obj
 0003:0001198c       ?useSurroundSound@@3HA     0043098c   M1Dlg.obj
 0003:00011990       ?curtime@@3PADA            00430990   M1Dlg.obj
 0003:0001199c       ?useVolumeBars@@3HA        0043099c   M1Dlg.obj
 0003:000119a0       ?mds@@3PAVMyDsound@@A      004309a0   M1Dlg.obj
 0003:000119a4       ?myhwnd@@3PAUHWND__@@A     004309a4   M1Dlg.obj
 0003:000119a8       ?pdViewable@@3HA           004309a8   M1Dlg.obj
 0003:000119ac       ?md@@3PAVCM1Dlg@@A         004309ac   M1Dlg.obj
 0003:000119b0       ?od@@3PAVCOptionsDlg@@A    004309b0   M1Dlg.obj
 0003:000119b4       ?pd@@3PAVCPlaylistDlg@@A   004309b4   M1Dlg.obj
 0003:000119b8       ?threadID@@3KA             004309b8   M1Dlg.obj
 0003:000119bc       ?threadHandle@@3PAXA       004309bc   M1Dlg.obj
 0003:000119c0       ?stereo@@3HA               004309c0   M1Dlg.obj
 0003:000119c4       ?hertz@@3JA                004309c4   M1Dlg.obj
 0003:000119cc       ?odViewable@@3HA           004309cc   M1Dlg.obj
 0003:000119d0       ?myFont@@3VCFont@@A        004309d0   M1Dlg.obj
 0003:000119d8       ?icoSkipb@@3PAUHICON__@@A  004309d8   M1.obj
 0003:000119dc       ?icoSkipf@@3PAUHICON__@@A  004309dc   M1.obj
 0003:000119e0       ?icoPlay@@3PAUHICON__@@A   004309e0   M1.obj
 0003:000119e4       ?icoPlayOn@@3PAUHICON__@@A 004309e4   M1.obj
 0003:000119e8       ?icoOption@@3PAUHICON__@@A 004309e8   M1.obj
 0003:000119ec       ?icoStop@@3PAUHICON__@@A   004309ec   M1.obj
 0003:000119f0       ?icoFf@@3PAUHICON__@@A     004309f0   M1.obj
 0003:000119f4       ?icoRw@@3PAUHICON__@@A     004309f4   M1.obj
 0003:000119f8       ?theApp@@3VCM1App@@A       004309f8   M1.obj
 0003:00011ac0       __afxForceEXCLUDE          00430ac0   mfcs40d:nolib.obj
 0003:00011ac4       __afxForceSTDAFX           00430ac4   mfcs40d:stdafx.obj
 0003:00011ac8       ?_afxTermAppState@@3V_AFX_TERM_APP_STATE@@A 00430ac8   mfcs40d:appmodul.obj
 0003:00011acc       ___onexitend               00430acc   <common>
 0003:00011ad0       ___onexitbegin             00430ad0   <common>
 0003:00011ad4       __adjust_fdiv              00430ad4   <common>
 0004:00000000       __IMPORT_DESCRIPTOR_DSOUND 00431000   dsound:DSOUND.dll
 0004:00000014       __IMPORT_DESCRIPTOR_MFC40D 00431014   mfc40d:MFC40D.DLL
 0004:00000028       __IMPORT_DESCRIPTOR_MSVCR40D 00431028   msvcrtd:MSVCR40D.dll
 0004:0000003c       __IMPORT_DESCRIPTOR_KERNEL32 0043103c   kernel32:KERNEL32.dll
 0004:00000050       __IMPORT_DESCRIPTOR_USER32 00431050   user32:USER32.dll
 0004:00000064       __IMPORT_DESCRIPTOR_SHELL32 00431064   shell32:SHELL32.dll
 0004:00000078       __NULL_IMPORT_DESCRIPTOR   00431078   dsound:DSOUND.dll
 0004:0000040c       __imp__DirectSoundCreate@12 0043140c   dsound:DSOUND.dll
 0004:00000410       \177DSOUND_NULL_THUNK_DATA 00431410   dsound:DSOUND.dll
 0004:00000414       __imp__SetThreadPriority@8 00431414   kernel32:KERNEL32.dll
 0004:00000418       __imp__Sleep@4             00431418   kernel32:KERNEL32.dll
 0004:0000041c       __imp__GetExitCodeThread@8 0043141c   kernel32:KERNEL32.dll
 0004:00000420       __imp__GetVersion@0        00431420   kernel32:KERNEL32.dll
 0004:00000424       __imp__GetModuleHandleA@4  00431424   kernel32:KERNEL32.dll
 0004:00000428       __imp__GetStartupInfoA@4   00431428   kernel32:KERNEL32.dll
 0004:0000042c       __imp__CreateThread@24     0043142c   kernel32:KERNEL32.dll
 0004:00000430       \177KERNEL32_NULL_THUNK_DATA 00431430   kernel32:KERNEL32.dll
 0004:00000434       __imp_?DefWindowProcA@CWnd@@MAEJIIJ@Z 00431434   mfc40d:MFC40D.DLL
 0004:00000438       __imp_?OnInitDialog@CDialog@@UAEHXZ 00431438   mfc40d:MFC40D.DLL
 0004:0000043c       __imp_?DoModal@CDialog@@UAEHXZ 0043143c   mfc40d:MFC40D.DLL
 0004:00000440       __imp_?SetOccDialogInfo@CDialog@@MAEHPAU_AFX_OCC_DIALOG_INFO@@@Z 00431440   mfc40d:MFC40D.DLL
 0004:00000444       __imp_?IsFrameWnd@CWnd@@UBEHXZ 00431444   mfc40d:MFC40D.DLL
 0004:00000448       __imp_?CheckAutoCenter@CDialog@@UAEHXZ 00431448   mfc40d:MFC40D.DLL
 0004:0000044c       __imp_?OnChildNotify@CWnd@@MAEHIIJPAJ@Z 0043144c   mfc40d:MFC40D.DLL
 0004:00000450       __imp_?OnOK@CDialog@@MAEXXZ 00431450   mfc40d:MFC40D.DLL
 0004:00000454       __imp_?OnSetFont@CDialog@@UAEXPAVCFont@@@Z 00431454   mfc40d:MFC40D.DLL
 0004:00000458       __imp_?OnWndMsg@CWnd@@MAEHIIJPAJ@Z 00431458   mfc40d:MFC40D.DLL
 0004:0000045c       __imp_?WindowProc@CWnd@@MAEJIIJ@Z 0043145c   mfc40d:MFC40D.DLL
 0004:00000460       __imp_?OnAmbientProperty@CWnd@@UAEHPAVCOleControlSite@@JPAUtagVARIANT@@@Z 00431460   mfc40d:MFC40D.DLL
 0004:00000464       __imp_?PreTranslateMessage@CDialog@@UAEHPAUtagMSG@@@Z 00431464   mfc40d:MFC40D.DLL
 0004:00000468       __imp_?EndModalState@CWnd@@UAEXXZ 00431468   mfc40d:MFC40D.DLL
 0004:0000046c       __imp_?BeginModalState@CWnd@@UAEXXZ 0043146c   mfc40d:MFC40D.DLL
 0004:00000470       __imp_?GetSuperWndProcAddr@CWnd@@MAEPAP6GJPAUHWND__@@IIJ@ZXZ 00431470   mfc40d:MFC40D.DLL
 0004:00000474       __imp_?PostNcDestroy@CWnd@@MAEXXZ 00431474   mfc40d:MFC40D.DLL
 0004:00000478       __imp_?OnNotify@CWnd@@MAEHIJPAJ@Z 00431478   mfc40d:MFC40D.DLL
 0004:0000047c       __imp_?EndModalLoop@CWnd@@UAEXH@Z 0043147c   mfc40d:MFC40D.DLL
 0004:00000480       __imp_?ContinueModal@CWnd@@UAEHXZ 00431480   mfc40d:MFC40D.DLL
 0004:00000484       __imp_?WinHelpA@CWnd@@UAEXKI@Z 00431484   mfc40d:MFC40D.DLL
 0004:00000488       __imp_?GetScrollBarCtrl@CWnd@@UBEPAVCScrollBar@@H@Z 00431488   mfc40d:MFC40D.DLL
 0004:0000048c       __imp_?OnToolHitTest@CWnd@@UBEHVCPoint@@PAUtagTOOLINFOA@@@Z 0043148c   mfc40d:MFC40D.DLL
 0004:00000490       __imp_?CalcWindowRect@CWnd@@UAEXPAUtagRECT@@I@Z 00431490   mfc40d:MFC40D.DLL
 0004:00000494       __imp_?PreCreateWindow@CWnd@@UAEHAAUtagCREATESTRUCTA@@@Z 00431494   mfc40d:MFC40D.DLL
 0004:00000498       __imp_?DestroyWindow@CWnd@@UAEHXZ 00431498   mfc40d:MFC40D.DLL
 0004:0000049c       __imp_?Create@CWnd@@UAEHPBD0KABUtagRECT@@PAV1@IPAUCCreateContext@@@Z 0043149c   mfc40d:MFC40D.DLL
 0004:000004a0       __imp_?PreSubclassWindow@CWnd@@UAEXXZ 004314a0   mfc40d:MFC40D.DLL
 0004:000004a4       __imp_?GetConnectionHook@CCmdTarget@@MAEPAUIConnectionPoint@@ABU_GUID@@@Z 004314a4   mfc40d:MFC40D.DLL
 0004:000004a8       __imp_?GetExtraConnectionPoints@CCmdTarget@@MAEHPAVCPtrArray@@@Z 004314a8   mfc40d:MFC40D.DLL
 0004:000004ac       __imp_?GetInterfaceHook@CCmdTarget@@UAEPAUIUnknown@@PBX@Z 004314ac   mfc40d:MFC40D.DLL
 0004:000004b0       __imp_?OnCreateAggregates@CCmdTarget@@UAEHXZ 004314b0   mfc40d:MFC40D.DLL
 0004:000004b4       __imp_?GetEventSinkMap@CCmdTarget@@MBEPBUAFX_EVENTSINKMAP@@XZ 004314b4   mfc40d:MFC40D.DLL
 0004:000004b8       __imp_?GetInterfaceMap@CCmdTarget@@MBEPBUAFX_INTERFACEMAP@@XZ 004314b8   mfc40d:MFC40D.DLL
 0004:000004bc       __imp_?GetConnectionMap@CCmdTarget@@MBEPBUAFX_CONNECTIONMAP@@XZ 004314bc   mfc40d:MFC40D.DLL
 0004:000004c0       __imp_?OnCommand@CWnd@@MAEHIJ@Z 004314c0   mfc40d:MFC40D.DLL
 0004:000004c4       __imp_?GetDispatchMap@CCmdTarget@@MBEPBUAFX_DISPMAP@@XZ 004314c4   mfc40d:MFC40D.DLL
 0004:000004c8       __imp_?GetTypeLibCache@CCmdTarget@@UAEPAVCTypeLibCache@@XZ 004314c8   mfc40d:MFC40D.DLL
 0004:000004cc       __imp_?GetTypeInfoCount@CCmdTarget@@UAEIXZ 004314cc   mfc40d:MFC40D.DLL
 0004:000004d0       __imp_?GetDispatchIID@CCmdTarget@@UAEHPAU_GUID@@@Z 004314d0   mfc40d:MFC40D.DLL
 0004:000004d4       __imp_?IsInvokeAllowed@CCmdTarget@@UAEHJ@Z 004314d4   mfc40d:MFC40D.DLL
 0004:000004d8       __imp_?OnFinalRelease@CWnd@@UAEXXZ 004314d8   mfc40d:MFC40D.DLL
 0004:000004dc       __imp_?OnCmdMsg@CDialog@@UAEHIHPAXPAUAFX_CMDHANDLERINFO@@@Z 004314dc   mfc40d:MFC40D.DLL
 0004:000004e0       __imp_?Dump@CDialog@@UBEXAAVCDumpContext@@@Z 004314e0   mfc40d:MFC40D.DLL
 0004:000004e4       __imp_?AssertValid@CDialog@@UBEXXZ 004314e4   mfc40d:MFC40D.DLL
 0004:000004e8       __imp_?Serialize@CObject@@UAEXAAVCArchive@@@Z 004314e8   mfc40d:MFC40D.DLL
 0004:000004ec       __imp_?GetRuntimeClass@CDialog@@UBEPAUCRuntimeClass@@XZ 004314ec   mfc40d:MFC40D.DLL
 0004:000004f0       __imp_??1CDialog@@UAE@XZ   004314f0   mfc40d:MFC40D.DLL
 0004:000004f4       __imp_??0CDialog@@QAE@IPAVCWnd@@@Z 004314f4   mfc40d:MFC40D.DLL
 0004:000004f8       __imp_??3CObject@@SGXPAX@Z 004314f8   mfc40d:MFC40D.DLL
 0004:000004fc       __imp_?DoDataExchange@CWnd@@MAEXPAVCDataExchange@@@Z 004314fc   mfc40d:MFC40D.DLL
 0004:00000500       __imp_?messageMap@CDialog@@1UAFX_MSGMAP@@B 00431500   mfc40d:MFC40D.DLL
 0004:00000504       __imp_?OnContextMenu@CWnd@@IAEXPAV1@VCPoint@@@Z 00431504   mfc40d:MFC40D.DLL
 0004:00000508       __imp_?SetIcon@CButton@@QAEPAUHICON__@@PAU2@@Z 00431508   mfc40d:MFC40D.DLL
 0004:0000050c       __imp_?SetWindowTextA@CWnd@@QAEXPBD@Z 0043150c   mfc40d:MFC40D.DLL
 0004:00000510       __imp_?KillTimer@CWnd@@QAEHH@Z 00431510   mfc40d:MFC40D.DLL
 0004:00000514       __imp_?SetTimer@CWnd@@QAEIIIP6GXPAUHWND__@@IIK@Z@Z 00431514   mfc40d:MFC40D.DLL
 0004:00000518       __imp_?GetBuffer@CString@@QAEPADH@Z 00431518   mfc40d:MFC40D.DLL
 0004:0000051c       __imp_??0CString@@QAE@PBD@Z 0043151c   mfc40d:MFC40D.DLL
 0004:00000520       __imp_??0CStdioFile@@QAE@PBDI@Z 00431520   mfc40d:MFC40D.DLL
 0004:00000524       __imp_??2CObject@@SGPAXI@Z 00431524   mfc40d:MFC40D.DLL
 0004:00000528       __imp_??0CFont@@QAE@XZ     00431528   mfc40d:MFC40D.DLL
 0004:0000052c       __imp_??1CFont@@UAE@XZ     0043152c   mfc40d:MFC40D.DLL
 0004:00000530       __imp_??1CStatic@@UAE@XZ   00431530   mfc40d:MFC40D.DLL
 0004:00000534       __imp_??1CButton@@UAE@XZ   00431534   mfc40d:MFC40D.DLL
 0004:00000538       __imp_?LoadIconA@CWinApp@@QBEPAUHICON__@@I@Z 00431538   mfc40d:MFC40D.DLL
 0004:0000053c       __imp_?AfxGetApp@@YGPAVCWinApp@@XZ 0043153c   mfc40d:MFC40D.DLL
 0004:00000540       __imp_??0CButton@@QAE@XZ   00431540   mfc40d:MFC40D.DLL
 0004:00000544       __imp_??0CStatic@@QAE@XZ   00431544   mfc40d:MFC40D.DLL
 0004:00000548       __imp_?DDX_Control@@YGXPAVCDataExchange@@HAAVCWnd@@@Z 00431548   mfc40d:MFC40D.DLL
 0004:0000054c       __imp_??1CString@@QAE@XZ   0043154c   mfc40d:MFC40D.DLL
 0004:00000550       __imp_?SetFont@CWnd@@QAEXPAVCFont@@H@Z 00431550   mfc40d:MFC40D.DLL
 0004:00000554       __imp_?CreatePointFont@CFont@@QAEHHPBDPAVCDC@@@Z 00431554   mfc40d:MFC40D.DLL
 0004:00000558       __imp_?GetTypeLib@CCmdTarget@@UAEJKPAPAUITypeLib@@@Z 00431558   mfc40d:MFC40D.DLL
 0004:0000055c       __imp_?PreInitDialog@CDialog@@MAEXXZ 0043155c   mfc40d:MFC40D.DLL
 0004:00000560       __imp_?OnCancel@CDialog@@MAEXXZ 00431560   mfc40d:MFC40D.DLL
 0004:00000564       __imp_??2CObject@@SGPAXIPBDH@Z 00431564   mfc40d:MFC40D.DLL
 0004:00000568       __imp_?SetIcon@CWnd@@QAEPAUHICON__@@PAU2@H@Z 00431568   mfc40d:MFC40D.DLL
 0004:0000056c       __imp_?AppendMenuA@CMenu@@QAEHIIPBD@Z 0043156c   mfc40d:MFC40D.DLL
 0004:00000570       __imp_??BCString@@QBEPBDXZ 00431570   mfc40d:MFC40D.DLL
 0004:00000574       __imp_?IsEmpty@CString@@QBEHXZ 00431574   mfc40d:MFC40D.DLL
 0004:00000578       __imp_?LoadStringA@CString@@QAEHI@Z 00431578   mfc40d:MFC40D.DLL
 0004:0000057c       __imp_??0CString@@QAE@XZ   0043157c   mfc40d:MFC40D.DLL
 0004:00000580       __imp_?GetSystemMenu@CWnd@@QBEPAVCMenu@@H@Z 00431580   mfc40d:MFC40D.DLL
 0004:00000584       __imp_?OnSysCommand@CWnd@@IAEXIJ@Z 00431584   mfc40d:MFC40D.DLL
 0004:00000588       __imp_??1CPaintDC@@UAE@XZ  00431588   mfc40d:MFC40D.DLL
 0004:0000058c       __imp_?OnPaint@CWnd@@IAEXXZ 0043158c   mfc40d:MFC40D.DLL
 0004:00000590       __imp_?DrawIcon@CDC@@QAEHHHPAUHICON__@@@Z 00431590   mfc40d:MFC40D.DLL
 0004:00000594       __imp_?Height@CRect@@QBEHXZ 00431594   mfc40d:MFC40D.DLL
 0004:00000598       __imp_?Width@CRect@@QBEHXZ 00431598   mfc40d:MFC40D.DLL
 0004:0000059c       __imp_?GetClientRect@CWnd@@QBEXPAUtagRECT@@@Z 0043159c   mfc40d:MFC40D.DLL
 0004:000005a0       __imp_??0CRect@@QAE@XZ     004315a0   mfc40d:MFC40D.DLL
 0004:000005a4       __imp_?SendMessageA@CWnd@@QAEJIIJ@Z 004315a4   mfc40d:MFC40D.DLL
 0004:000005a8       __imp_?GetSafeHdc@CDC@@QBEPAUHDC__@@XZ 004315a8   mfc40d:MFC40D.DLL
 0004:000005ac       __imp_??0CPaintDC@@QAE@PAVCWnd@@@Z 004315ac   mfc40d:MFC40D.DLL
 0004:000005b0       __imp_?IsIconic@CWnd@@QBEHXZ 004315b0   mfc40d:MFC40D.DLL
 0004:000005b4       __imp_?GetCheck@CButton@@QBEHXZ 004315b4   mfc40d:MFC40D.DLL
 0004:000005b8       __imp_?SetFocus@CWnd@@QAEPAV1@XZ 004315b8   mfc40d:MFC40D.DLL
 0004:000005bc       __imp_?SetForegroundWindow@CWnd@@QAEHXZ 004315bc   mfc40d:MFC40D.DLL
 0004:000005c0       __imp_??2@YAPAXIPBDH@Z     004315c0   mfc40d:MFC40D.DLL
 0004:000005c4       __imp_?SetWindowPos@CWnd@@QAEHPBV1@HHHHI@Z 004315c4   mfc40d:MFC40D.DLL
 0004:000005c8       __imp_?GetWindowPlacement@CWnd@@QBEHPAUtagWINDOWPLACEMENT@@@Z 004315c8   mfc40d:MFC40D.DLL
 0004:000005cc       __imp_??3@YAXPAX@Z         004315cc   mfc40d:MFC40D.DLL
 0004:000005d0       __imp_?GetRuntimeClass@CObject@@UBEPAUCRuntimeClass@@XZ 004315d0   mfc40d:MFC40D.DLL
 0004:000005d4       __imp_??1CObject@@UAE@XZ   004315d4   mfc40d:MFC40D.DLL
 0004:000005d8       __imp_??0CObject@@IAE@XZ   004315d8   mfc40d:MFC40D.DLL
 0004:000005dc       __imp_?AfxAssertValidObject@@YGXPBVCObject@@PBDH@Z 004315dc   mfc40d:MFC40D.DLL
 0004:000005e0       __imp_?ReadCount@CArchive@@QAEKXZ 004315e0   mfc40d:MFC40D.DLL
 0004:000005e4       __imp_?WriteCount@CArchive@@QAEXK@Z 004315e4   mfc40d:MFC40D.DLL
 0004:000005e8       __imp_?IsStoring@CArchive@@QBEHXZ 004315e8   mfc40d:MFC40D.DLL
 0004:000005ec       __imp_??6CDumpContext@@QAEAAV0@PBD@Z 004315ec   mfc40d:MFC40D.DLL
 0004:000005f0       __imp_?GetDepth@CDumpContext@@QBEHXZ 004315f0   mfc40d:MFC40D.DLL
 0004:000005f4       __imp_??6CDumpContext@@QAEAAV0@H@Z 004315f4   mfc40d:MFC40D.DLL
 0004:000005f8       __imp_?Dump@CObject@@UBEXAAVCDumpContext@@@Z 004315f8   mfc40d:MFC40D.DLL
 0004:000005fc       __imp_?AfxAssertFailedLine@@YGHPBDH@Z 004315fc   mfc40d:MFC40D.DLL
 0004:00000600       __imp_?AfxIsValidAddress@@YGHPBXIH@Z 00431600   mfc40d:MFC40D.DLL
 0004:00000604       __imp_?AssertValid@CObject@@UBEXXZ 00431604   mfc40d:MFC40D.DLL
 0004:00000608       __imp_?Read@CArchive@@QAEIPAXI@Z 00431608   mfc40d:MFC40D.DLL
 0004:0000060c       __imp_?Write@CArchive@@QAEXPBXI@Z 0043160c   mfc40d:MFC40D.DLL
 0004:00000610       __imp_?OnHelp@CWinApp@@IAEXXZ 00431610   mfc40d:MFC40D.DLL
 0004:00000614       __imp_?messageMap@CWinApp@@1UAFX_MSGMAP@@B 00431614   mfc40d:MFC40D.DLL
 0004:00000618       __imp_?WinHelpA@CWinApp@@UAEXKI@Z 00431618   mfc40d:MFC40D.DLL
 0004:0000061c       __imp_?OnDDECommand@CWinApp@@UAEHPAD@Z 0043161c   mfc40d:MFC40D.DLL
 0004:00000620       __imp_?DoWaitCursor@CWinApp@@UAEXH@Z 00431620   mfc40d:MFC40D.DLL
 0004:00000624       __imp_?DoMessageBox@CWinApp@@UAEHPBDII@Z 00431624   mfc40d:MFC40D.DLL
 0004:00000628       __imp_?SaveAllModified@CWinApp@@UAEHXZ 00431628   mfc40d:MFC40D.DLL
 0004:0000062c       __imp_?InitApplication@CWinApp@@UAEHXZ 0043162c   mfc40d:MFC40D.DLL
 0004:00000630       __imp_?AddToRecentFileList@CWinApp@@UAEXPBD@Z 00431630   mfc40d:MFC40D.DLL
 0004:00000634       __imp_?OpenDocumentFile@CWinApp@@UAEPAVCDocument@@PBD@Z 00431634   mfc40d:MFC40D.DLL
 0004:00000638       __imp_?Delete@CWinThread@@UAEXXZ 00431638   mfc40d:MFC40D.DLL
 0004:0000063c       __imp_?GetMainWnd@CWinThread@@UAEPAVCWnd@@XZ 0043163c   mfc40d:MFC40D.DLL
 0004:00000640       __imp_?ProcessMessageFilter@CWinThread@@UAEHHPAUtagMSG@@@Z 00431640   mfc40d:MFC40D.DLL
 0004:00000644       __imp_?ProcessWndProcException@CWinApp@@UAEJPAVCException@@PBUtagMSG@@@Z 00431644   mfc40d:MFC40D.DLL
 0004:00000648       __imp_?ExitInstance@CWinApp@@UAEHXZ 00431648   mfc40d:MFC40D.DLL
 0004:0000064c       __imp_?IsIdleMessage@CWinThread@@UAEHPAUtagMSG@@@Z 0043164c   mfc40d:MFC40D.DLL
 0004:00000650       __imp_?OnIdle@CWinApp@@UAEHJ@Z 00431650   mfc40d:MFC40D.DLL
 0004:00000654       __imp_?PumpMessage@CWinThread@@UAEHXZ 00431654   mfc40d:MFC40D.DLL
 0004:00000658       __imp_?PreTranslateMessage@CWinThread@@UAEHPAUtagMSG@@@Z 00431658   mfc40d:MFC40D.DLL
 0004:0000065c       __imp_?Run@CWinApp@@UAEHXZ 0043165c   mfc40d:MFC40D.DLL
 0004:00000660       __imp_?OnFinalRelease@CCmdTarget@@UAEXXZ 00431660   mfc40d:MFC40D.DLL
 0004:00000664       __imp_?OnCmdMsg@CCmdTarget@@UAEHIHPAXPAUAFX_CMDHANDLERINFO@@@Z 00431664   mfc40d:MFC40D.DLL
 0004:00000668       __imp_?Dump@CWinApp@@UBEXAAVCDumpContext@@@Z 00431668   mfc40d:MFC40D.DLL
 0004:0000066c       __imp_?AssertValid@CWinApp@@UBEXXZ 0043166c   mfc40d:MFC40D.DLL
 0004:00000670       __imp_?GetRuntimeClass@CWinApp@@UBEPAUCRuntimeClass@@XZ 00431670   mfc40d:MFC40D.DLL
 0004:00000674       __imp_??1CWinApp@@UAE@XZ   00431674   mfc40d:MFC40D.DLL
 0004:00000678       __imp_??0CWinApp@@QAE@PBD@Z 00431678   mfc40d:MFC40D.DLL
 0004:0000067c       __imp_?Enable3dControls@CWinApp@@IAEHXZ 0043167c   mfc40d:MFC40D.DLL
 0004:00000680       __imp_?SetDialogBkColor@CWinApp@@IAEXKK@Z 00431680   mfc40d:MFC40D.DLL
 0004:00000684       __imp_??1CSliderCtrl@@UAE@XZ 00431684   mfc40d:MFC40D.DLL
 0004:00000688       __imp_??0CSliderCtrl@@QAE@XZ 00431688   mfc40d:MFC40D.DLL
 0004:0000068c       __imp_?GetPos@CSliderCtrl@@QBEHXZ 0043168c   mfc40d:MFC40D.DLL
 0004:00000690       __imp_?SetRange@CSliderCtrl@@QAEXHHH@Z 00431690   mfc40d:MFC40D.DLL
 0004:00000694       __imp_?SetPos@CSliderCtrl@@QAEXH@Z 00431694   mfc40d:MFC40D.DLL
 0004:00000698       __imp_??2@YAPAXI@Z         00431698   mfc40d:MFC40D.DLL
 0004:0000069c       __imp_?Create@CDialog@@QAEHIPAVCWnd@@@Z 0043169c   mfc40d:MFC40D.DLL
 0004:000006a0       __imp_?DragAcceptFiles@CWnd@@QAEXH@Z 004316a0   mfc40d:MFC40D.DLL
 0004:000006a4       __imp_?GetSafeHwnd@CWnd@@QBEPAUHWND__@@XZ 004316a4   mfc40d:MFC40D.DLL
 0004:000006a8       __imp_?ShowWindow@CWnd@@QAEHH@Z 004316a8   mfc40d:MFC40D.DLL
 0004:000006ac       __imp_?AfxWinMain@@YGHPAUHINSTANCE__@@0PADH@Z 004316ac   mfc40d:MFC40D.DLL
 0004:000006b0       __imp_?AfxGetModuleState@@YGPAVAFX_MODULE_STATE@@XZ 004316b0   mfc40d:MFC40D.DLL
 0004:000006b4       \177MFC40D_NULL_THUNK_DATA 004316b4   mfc40d:MFC40D.DLL
 0004:000006b8       __imp__sin                 004316b8   msvcrtd:MSVCR40D.dll
 0004:000006bc       __imp___adj_fdivr_m32      004316bc   msvcrtd:MSVCR40D.dll
 0004:000006c0       __imp___adj_fdiv_m64       004316c0   msvcrtd:MSVCR40D.dll
 0004:000006c4       __imp__pow                 004316c4   msvcrtd:MSVCR40D.dll
 0004:000006c8       __imp__memcpy              004316c8   msvcrtd:MSVCR40D.dll
 0004:000006cc       __imp__putc                004316cc   msvcrtd:MSVCR40D.dll
 0004:000006d0       __imp__memset              004316d0   msvcrtd:MSVCR40D.dll
 0004:000006d4       __imp___ftol               004316d4   msvcrtd:MSVCR40D.dll
 0004:000006d8       __imp__sqrt                004316d8   msvcrtd:MSVCR40D.dll
 0004:000006dc       __imp__log                 004316dc   msvcrtd:MSVCR40D.dll
 0004:000006e0       __imp___itoa               004316e0   msvcrtd:MSVCR40D.dll
 0004:000006e4       __imp__abs                 004316e4   msvcrtd:MSVCR40D.dll
 0004:000006e8       __imp__strrchr             004316e8   msvcrtd:MSVCR40D.dll
 0004:000006ec       __imp__strlen              004316ec   msvcrtd:MSVCR40D.dll
 0004:000006f0       __imp__strstr              004316f0   msvcrtd:MSVCR40D.dll
 0004:000006f4       __imp__fprintf             004316f4   msvcrtd:MSVCR40D.dll
 0004:000006f8       __imp__malloc              004316f8   msvcrtd:MSVCR40D.dll
 0004:000006fc       __imp____dllonexit         004316fc   msvcrtd:MSVCR40D.dll
 0004:00000700       __imp___onexit             00431700   msvcrtd:MSVCR40D.dll
 0004:00000704       __imp__strcpy              00431704   msvcrtd:MSVCR40D.dll
 0004:00000708       __imp___exit               00431708   msvcrtd:MSVCR40D.dll
 0004:0000070c       __imp__exit                0043170c   msvcrtd:MSVCR40D.dll
 0004:00000710       __imp____p__acmdln         00431710   msvcrtd:MSVCR40D.dll
 0004:00000714       __imp___initterm           00431714   msvcrtd:MSVCR40D.dll
 0004:00000718       __imp____getmainargs       00431718   msvcrtd:MSVCR40D.dll
 0004:0000071c       __imp__cos                 0043171c   msvcrtd:MSVCR40D.dll
 0004:00000720       __imp___adjust_fdiv        00431720   msvcrtd:MSVCR40D.dll
 0004:00000724       __imp____p__commode        00431724   msvcrtd:MSVCR40D.dll
 0004:00000728       __imp____p__fmode          00431728   msvcrtd:MSVCR40D.dll
 0004:0000072c       __imp____set_app_type      0043172c   msvcrtd:MSVCR40D.dll
 0004:00000730       __imp___except_handler3    00431730   msvcrtd:MSVCR40D.dll
 0004:00000734       __imp___controlfp          00431734   msvcrtd:MSVCR40D.dll
 0004:00000738       __imp___adj_fdivr_m64      00431738   msvcrtd:MSVCR40D.dll
 0004:0000073c       __imp___purecall           0043173c   msvcrtd:MSVCR40D.dll
 0004:00000740       __imp____CxxFrameHandler   00431740   msvcrtd:MSVCR40D.dll
 0004:00000744       __imp__fread               00431744   msvcrtd:MSVCR40D.dll
 0004:00000748       __imp__getc                00431748   msvcrtd:MSVCR40D.dll
 0004:0000074c       __imp__fclose              0043174c   msvcrtd:MSVCR40D.dll
 0004:00000750       __imp____p__iob            00431750   msvcrtd:MSVCR40D.dll
 0004:00000754       __imp__fopen               00431754   msvcrtd:MSVCR40D.dll
 0004:00000758       __imp___XcptFilter         00431758   msvcrtd:MSVCR40D.dll
 0004:0000075c       __imp____setusermatherr    0043175c   msvcrtd:MSVCR40D.dll
 0004:00000760       __imp___open               00431760   msvcrtd:MSVCR40D.dll
 0004:00000760       __imp__open                00431760   msvcrtd:MSVCR40D.dll
 0004:00000764       __imp___read               00431764   msvcrtd:MSVCR40D.dll
 0004:00000764       __imp__read                00431764   msvcrtd:MSVCR40D.dll
 0004:00000768       __imp___close              00431768   msvcrtd:MSVCR40D.dll
 0004:00000768       __imp__close               00431768   msvcrtd:MSVCR40D.dll
 0004:0000076c       __imp___write              0043176c   msvcrtd:MSVCR40D.dll
 0004:0000076c       __imp__write               0043176c   msvcrtd:MSVCR40D.dll
 0004:00000770       __imp___setmbcp            00431770   msvcrtd:MSVCR40D.dll
 0004:00000774       \177MSVCR40D_NULL_THUNK_DATA 00431774   msvcrtd:MSVCR40D.dll
 0004:00000778       __imp__DragQueryFileA@16   00431778   shell32:SHELL32.dll
 0004:0000077c       \177SHELL32_NULL_THUNK_DATA 0043177c   shell32:SHELL32.dll
 0004:00000780       __imp__GetSystemMetrics@4  00431780   user32:USER32.dll
 0004:00000784       __imp__MessageBoxA@16      00431784   user32:USER32.dll
 0004:00000788       \177USER32_NULL_THUNK_DATA 00431788   user32:USER32.dll

 entry point at        0001:00015dc0

 Static symbols

 0001:00012951       _$E186                     00413951 f M1.obj
 0001:0001296b       _$E183                     0041396b f M1.obj
 0001:00012985       _$E185                     00413985 f M1.obj
 0001:000129a2       _$E184                     004139a2 f M1.obj
 0001:0000f0de       _$E225                     004100de f M1Dlg.obj
 0001:0000f0f8       _$E222                     004100f8 f M1Dlg.obj
 0001:0000f112       _$E224                     00410112 f M1Dlg.obj
 0001:0000f12f       _$E223                     0041012f f M1Dlg.obj
 0001:00000500       _$E215                     00401500 f filter.obj
 0001:00000515       _$E214                     00401515 f filter.obj
 0001:00000589       _$E218                     00401589 f filter.obj
 0001:0000059e       _$E217                     0040159e f filter.obj
 0001:00000618       _$E221                     00401618 f filter.obj
 0001:0000062d       _$E220                     0040162d f filter.obj
 0001:000006a7       _$E224                     004016a7 f filter.obj
 0001:000006bc       _$E223                     004016bc f filter.obj
 0001:00000736       _$E227                     00401736 f filter.obj
 0001:0000074b       _$E226                     0040174b f filter.obj
 0001:000007c5       _$E230                     004017c5 f filter.obj
 0001:000007da       _$E229                     004017da f filter.obj
 0001:00000854       _$E233                     00401854 f filter.obj
 0001:00000869       _$E232                     00401869 f filter.obj
 0001:000008e3       _$E236                     004018e3 f filter.obj
 0001:000008f8       _$E235                     004018f8 f filter.obj
 0001:00000972       _$E239                     00401972 f filter.obj
 0001:00000987       _$E238                     00401987 f filter.obj
 0001:00000a01       _$E242                     00401a01 f filter.obj
 0001:00000a16       _$E241                     00401a16 f filter.obj
 0001:00000a90       _$E245                     00401a90 f filter.obj
 0001:00000aa5       _$E244                     00401aa5 f filter.obj
 0001:00000b1f       _$E248                     00401b1f f filter.obj
 0001:00000b34       _$E247                     00401b34 f filter.obj
 0001:00000bae       _$E251                     00401bae f filter.obj
 0001:00000bc3       _$E250                     00401bc3 f filter.obj
 0001:00000c3d       _$E254                     00401c3d f filter.obj
 0001:00000c52       _$E253                     00401c52 f filter.obj
 0001:00000ccc       _$E257                     00401ccc f filter.obj
 0001:00000ce1       _$E256                     00401ce1 f filter.obj
 0001:00000d5b       _$E260                     00401d5b f filter.obj
 0001:00000d70       _$E259                     00401d70 f filter.obj
 0001:00000dea       _$E263                     00401dea f filter.obj
 0001:00000dff       _$E262                     00401dff f filter.obj
 0001:00000e73       _$E266                     00401e73 f filter.obj
 0001:00000e88       _$E265                     00401e88 f filter.obj
 0001:00000f02       _$E269                     00401f02 f filter.obj
 0001:00000f17       _$E268                     00401f17 f filter.obj
 0001:00000f91       _$E272                     00401f91 f filter.obj
 0001:00000fa6       _$E271                     00401fa6 f filter.obj
 0001:00001020       _$E275                     00402020 f filter.obj
 0001:00001035       _$E274                     00402035 f filter.obj
 0001:000010af       _$E278                     004020af f filter.obj
 0001:000010c4       _$E277                     004020c4 f filter.obj
 0001:0000113e       _$E281                     0040213e f filter.obj
 0001:00001153       _$E280                     00402153 f filter.obj
 0001:000011cd       _$E284                     004021cd f filter.obj
 0001:000011e2       _$E283                     004021e2 f filter.obj
 0001:0000125c       _$E287                     0040225c f filter.obj
 0001:00001271       _$E286                     00402271 f filter.obj
 0001:000012e5       _$E290                     004022e5 f filter.obj
 0001:000012fa       _$E289                     004022fa f filter.obj
 0001:00001374       _$E293                     00402374 f filter.obj
 0001:00001389       _$E292                     00402389 f filter.obj
 0001:00001403       _$E296                     00402403 f filter.obj
 0001:00001418       _$E295                     00402418 f filter.obj
 0001:00001492       _$E299                     00402492 f filter.obj
 0001:000014a7       _$E298                     004024a7 f filter.obj
 0001:0000151b       _$E302                     0040251b f filter.obj
 0001:00001530       _$E301                     00402530 f filter.obj
 0001:000015aa       _$E305                     004025aa f filter.obj
 0001:000015bf       _$E304                     004025bf f filter.obj
 0001:000161c0       _$E321                     004171c0 f mfcs40d:appmodul.obj
 0001:000161e0       _$E320                     004171e0 f mfcs40d:appmodul.obj
 0001:00015c40       _$$$00001                  00416c40 f msvcrtd:chkstk.obj

FIXUPS: 16fc9 fffffd8d 35 ffff1cc8 3c 2e4 3c e 3c 2e4 3c e 3c ffff81ab
FIXUPS: 1319 2e 37 8d 65 13 4d 13 fffffd27 15efd 23 25 55 23 25 fffffe55
FIXUPS: 16e42 20 f 39 e6 fffeff73 3c 2e4 3c e 3c 2e4 3c e 3c 2e4 3c e 3c
FIXUPS: 7c61 3c e 3c 2e4 3c e 3c 2e4 3c e 3c 2e4 3c e 3c 2e4 3c ffffc79f
FIXUPS: 5220 1a4 3c 1a4 3c 1a4 3c 1a4 3c 407 3c e 3c 2e4 3c e 3c 2e4 3c
FIXUPS: 64c5 3c 2e4 3c e 3c 2e4 3c e 3c 2e4 3c ffffb676 2b 1b 38 b 2b 14c1
FIXUPS: 3af5 1a 8 22d 3c 1a4 3c 1a4 3c 1a4 3c 1a4 3c 1a4 3c 1a4 3c 1a4
FIXUPS: 4aa0 1a4 3c 1a4 3c 1a4 3c ffffd0bf 2b 1b 3e b 2b 1b 3e b 2b 1b
FIXUPS: 229b b 2b 1b 3e b 2b 1b 3e b 2b 1b 3e b 2b 1b 38 b 2b 1b 3e fffff72d
FIXUPS: 1cb8 1b 3e b 2b 1b 3e b 2b 1b 38 b 2b 1b 3e b 2b 1b 3e b 2b 1b
FIXUPS: 1fd6 b 2b 1b 3e b 2b 1b 3e fffff721 2b 1b 3e b 2b 1b 3e b 2b 1b
FIXUPS: 19b7 b 2b 1b 3e b 2b 1b 3e b 2b 1b 3e b 2b 1b 3e b 2b 1b 3e b81a
FIXUPS: d4ac 10 10 18 e e a9 d7 c2b ffff325c 38 b 2b 1b 3e b 2b 1b 3e b
FIXUPS: 1693 1b 3e b 2b 1b 3e b 2b 1b 3e a538 1d 1f 55 34 5a 41a 6f f48
FIXUPS: d252 18 11 11 11 11 1e 11 11 11 62 10 10 10 e 1d e 10 10 10 10
FIXUPS: d41a 72 ffffd358 2bd 10c 15b 148 2de 452 a7 17 13c 81 23 1e 20
FIXUPS: b90c 1fe 1c 14 2b 12 16 17 2a 4e 39 2a 1a 18 1f 21 1a 18 ffffe597
FIXUPS: a2cf 15 15 15 71 11 12 12 12 12 38 12 12 12 12 38 12 12 12 12 38
FIXUPS: a522 12 12 12 168 45 25 57 12 3f fffff82d 4b 12 15 15 12 15 15
FIXUPS: a0d4 15 15 12 15 15 12 15 15 12 15 15 12 15 15 12 15 15 12 15 15
FIXUPS: a27b 15 15 fffffade 12 12 12 12 12 12 12 15 15 12 15 15 12 15 15
FIXUPS: 9eb5 15 15 12 15 15 12 15 15 15 15 15 15 15 15 15 5044 5b 2d 5a
FIXUPS: f155 9b 9 10 2a 25 b 18 1c a 2a fffff0c9 79 ffffae72 4e 59 6d 9e
FIXUPS: 949a 22 66 4b 77 a3 77 59f c3 11 825d 14 3f 14 1b 2a ffffd4f4 2c
FIXUPS: f5a5 29 52 13 5f b ffffee43 2b 45 6f 19d 1a6 27 1d4 27 1e2 d 4a
FIXUPS: ed9e 92 23 7a bc 2d 2a41 21 17 31 13 38 19 46 18 51 1f 19 57 30
FIXUPS: 11cd8 25 1f 20 21 25 18 66 4b 19 27 46 14 59 14 11 1b 18 fffff659
FIXUPS: 115fa 3b 58 b 59 33 5c 20 18 21 b 37 c 8 17 d 11 17 29 19 7 7 8
FIXUPS: 118e8 17 d 24 29 25 2a 25 fffff6a8 2c b b4 13 34 59 13 8c 21 b
FIXUPS: 112f0 13 66 27 13 5f b 23 13 101 f f f f f f f f f f c fffff43c
FIXUPS: 10a3e d b 4e 8 27 46 13 5f 13 5a 13 81 13 50 2d 27 15 b 8 27 46
FIXUPS: 10deb db 4e 12 11 39 32 22 72 fffff6f8 13 1c 1e 14 14 14 14 14
FIXUPS: 107f3 13 16 15 10 13 13 13 23 b 49 f 21 d b 3f 17 11 e 1e f 8 15
FIXUPS: 10407 b 29 15 17 17 17 17 14 17 17 17 17 17 17 65 16 b 11 8 19
FIXUPS: 1060a d 14 14 14 17 25 17 28 14 1c fffffa3d 37 2c b 27 6b 12 12
FIXUPS: 10271 12 12 12 12 12 12 12 12 12 17 7 2b f f f f f f f f f f c
FIXUPS: fc01 17 31 38 b 31 60 e e3 78 11 18 a 22 3c 20 25 3f 1c 7 10 12
FIXUPS: fffd 82 2c d 9 b 19 5 1a 1a 2a75 21 eb 8f 4f 4f d1 8f 4f 4f e3
FIXUPS: 1318a 69 69 639 ffffbef6 2d 1a7 e 4f 17 30 17 3d f 3c 14 13 28
FIXUPS: fb65 42 b 3ecd 15 15 10 d 21 48 b 26 13 5f b ffffe568 21 4a 84
FIXUPS: 12262 5f 31f 21 21 26 3b 26 5a 21 358 21 21 23 3b 23 21a4 3a 7a
FIXUPS: 14dc3 60 4d 13 7a 23 b 25 13 73 ffffec75 b 62 b8 13 fffffb84 2c
FIXUPS: 1393e 1a 5 1a 1a 1d 58 10 15 15 15 15 a20 c 13 2e 48 59 26 26 2f
FIXUPS: 1464d 1b 48 175 2c b 69 2c b 59 36 b 7a 13 30 b4 1f 6f 2a e 86
FIXUPS: 14c87 2c fffff366 59 10 e d d d e 28 3f 1b 74 1f 41 1f 36 30 9
FIXUPS: 142b5 1f 59 3f f 2d 59 10 10 d d d e 28 1277 14e 22 22 22 51 15
FIXUPS: 1594b 15 66 fffff7cb 1a 37 7f 35 5e 95 40 5d 22e ffffe7c4 1f 41
FIXUPS: 13e97 36 30 9 40 1b 26 59 c 26ee fffff75b e0 81 320 55 25 45 39
FIXUPS: 16408 19 19 35 b 10 9 fffff5db 12 12 2f c 9 b 29 15 17 5a 13 7f
FIXUPS: 15c2e 9 b
